:020000040800F2
:10000000807B0020610200085D4D0008E34100088C
:10001000594D000881080008295900080000000017
:10002000000000000000000000000000A101000826
:100030002F0A000800000000FD010008BD4E000866
:100040007B0200087B0200087B0200087B0200089C
:100050007B0200087B0200087B0200087B0200088C
:100060007B0200087B0200087B0200087B0200087C
:100070007B0200087B020008D5080008E50800089C
:100080007B0200087B0200087B0200087B0200085C
:100090007B0200087B0200087B0200087B0200084C
:1000A000B94F0008D14F00087B0200087B0200080E
:1000B0007B0200087B020008E94F00087B02000871
:1000C0007B0200087B0200087B0200087B0200081C
:1000D0007B0200087B02000801590008155900083E
:1000E0007B0200087B0200087B0200087B020008FC
:1000F0007B0200087B0200087B0200087B020008EC
:100100007B0200087B0200087B0200087B020008DB
:10011000355400087B020008215000087B020008CB
:10012000F508000805090008150900087B02000809
:100130007B0200087B0200087B0200087B020008AB
:100140007B0200087B0200087B0200087B0200089B
:100150007B0200087B0200087B0200087B0200088B
:100160007B0200087B0200087B0200087B0200087B
:100170007B0200087B0200087B02000800000000F0
:100180007B0200087B020008DFF810D000F062FA62
:100190000048004701870008AFF30080807B002003
:1001A0002C4B19680868B0E8F04F80F30988BFF35A
:1001B0006F8F4FF0000080F311887047000000003F
:1001C00008480068006880F308884FF0000080F35A
:1001D000148862B661B6BFF34F8FBFF36F8F00DF35
:1001E00000BF00BF08ED00E0DFF80C00016841F43B
:1001F00070010160704700BF88ED00E0EFF30980F7
:10020000BFF36F8F134B1A681EF0100F08BF20ED5D
:10021000108A20E9F04F106009B44FF0500080F3CD
:100220001188BFF34F8FBFF36F8F09F061F94FF063
:10023000000080F3118809BC19680868B0E8F04F25
:100240001EF0100F08BFB0EC108A80F30988BFF3CE
:100250006F8F704730000020EFF30580704700007B
:100260000648804706480047FEE7FEE7FEE7FEE750
:10027000FEE7FEE7FEE7FEE7FEE7FEE7A54F000824
:10028000890100082DE9F05F0546002092469B4653
:1002900088460646814640241BE02846414647469C
:1002A000224600F032F953465A46C01A914110D303
:1002B00011461846224600F019F92D1A67EB01087D
:1002C0004F4622460120002100F010F917EB0009EB
:1002D0004E41201EA4F10104DFDC484631462A4687
:1002E0004346BDE8F09F40EA01039B0703D009E0C5
:1002F00008C9121F08C0042AFAD203E011F8013B12
:1003000000F8013B521EF9D27047D2B201E000F86A
:10031000012B491EFBD270470022F6E710B51346A9
:100320000A4604461946FFF7F0FF204610BD2DE9A6
:10033000FE4F81EA030404F0004421F000410094E0
:100340004FF0000B23F0004350EA01045ED052EA64
:1003500003045BD0C3F30A54C1F30A552C44A4F23E
:10036000F3340194A0FB0254C1F3130141F4801152
:10037000C3F3130343F4801301FB024400FB034E59
:10038000840A970A44EA815447EA8357A4FB076822
:1003900002958D0A05FB07854FEA932C04FB0C544C
:1003A0002705029D4FEA065847EA1637B5EB0805C0
:1003B0006EEB070C870E920E47EA811742EA831212
:1003C000A7FB0201B6EB0B0164EB00042B0D43EA23
:1003D0000C335E1844EB1C50DA465146E7FB020131
:1003E000C5F313044FEA0B3343EA14534FEA0432C4
:1003F000019C43EA0603A4F10C040294009CCDE99D
:1004000000B400F0D8F803B0BDE8F08F002001463A
:10041000F9E70EB540F2334102910021CDE9001118
:100420000A460B4600F0C7F803B000BD00F00042DA
:1004300030F000400AD0C10D01F56071C0F3160024
:1004400042EA0151C20840071143704700200146AB
:100450007047000030B5041E71F1000404DB4FF05A
:100460000044404264EB0101141E73F1000405DBFB
:100470001C464FF00043524263EB04038B4208BF1B
:10048000824230BD30B5041E71F1000404DB4FF030
:100490000044404264EB0101141E73F1000405DBCB
:1004A0001C464FF00043524263EB0403994208BFDD
:1004B000904230BD01F0004330B421F0004150EAD9
:1004C000010206D00A0DA2F56072C1F31301002AE1
:1004D00002DC30BC00207047440F44EAC104C10074
:1004E000E01830BC00EBC25000F01FB8202A04DB3B
:1004F000203A00FA02F1002070479140C2F1200337
:1005000020FA03F3194390407047202A04DB203A75
:1005100021FA02F00021704721FA02F3D040C2F123
:10052000200291400843194670470029A8BF704730
:10053000401C490008BF20F00100704710B4B0FA19
:1005400080FC00FA0CF050EA010404BF10BC7047B4
:1005500049B1CCF1200421FA04F411FA0CF118BFCE
:10056000012121430843A3EB0C01CB1D4FEA00619D
:100570004FEA102042BF002010BC704700EBC35070
:1005800010440029A4BF10BC7047401C490008BF9C
:1005900020F0010010BC704710B5141E73F1000468
:1005A00008DA401C41F1000192185B411A4301D165
:1005B00020F0010010BD2DE9F04D92469B4611B18F
:1005C000B1FA81F202E0B0FA80F220329046FFF7F1
:1005D0008DFF04460F4640EA0A0041EA0B015346EC
:1005E0005A46084313D0114653EA010019D0C8F106
:1005F00040025046FFF789FF05460E4650465946D1
:100600004246FFF773FF084305D0012004E020466F
:100610003946BDE8F08D0020054346EAE0762C43DC
:1006200037430A986305E40AA0EB08000022FD0A9C
:1006300044EA47540A3002D500200146E9E70105A3
:1006400010196941DDE9084500196941BDE8F04D1F
:10065000A2E70000064C074D06E0E06840F0010309
:1006600094E8070098471034AC42F6D3FFF790FDAA
:1006700030A1000850A1000870B50546AC6B206C95
:1006800000F0500050BB206C40F4007020642068E3
:10069000806800F04050E8B9207ED8B92068C06A70
:1006A00000F4700020B12068806800F4806088B990
:1006B0002068406820F0200021684860206C20F409
:1006C00080702064206C00F4805018B9206C40F0D9
:1006D00001002064204600F075FA0BE0206C00F069
:1006E000100018B1204600F06FFA03E0A06BC16C57
:1006F0002846884770BD70B50546AC6B4020206425
:10070000606C40F004006064204600F05DFA70BD4B
:1007100070B50446A56B284600F055FA70BD000080
:1007200055494A6822F440324A604A6843681A438D
:100730004A600268526822F4807203685A60026854
:100740005368026943EA022203685A6002685268E9
:1007500022F0407203685A600268526883681A4344
:1007600003685A600268926822F4006203689A6023
:1007700002689268C3681A4303689A603F4B826AB2
:100780009A4218D00268926822F0706203689A60F8
:1007900002689268836A1A4303689A6002689268E2
:1007A00022F0405203689A6002689268C36A1A4352
:1007B00003689A600BE00268926822F07062036836
:1007C0009A600268926822F0405203689A60026858
:1007D000926822F0020203689A6002689368027EBF
:1007E00043EA420203689A602022125CA2B10268C6
:1007F000526842F4006203685A600268526822F448
:10080000604203685A6002685368426A521E43EAB3
:10081000423203685A6005E00268526822F40062BE
:1008200003685A600268D26A22F470020368DA62CE
:100830000268D36A828B521E43EA02520368DA626C
:100840000268926822F4007203689A6002689368F2
:1008500090F8302043EA422203689A600268926866
:1008600022F4806203689A6002689368426943EAEE
:10087000822203689A607047002301400100000F44
:1008800000BFFEE730B502460D460AB9002030BD74
:100890000021002300244FF6FF7100BF12E0D05C5E
:1008A000414000240AE001F0010020B14AF20100B9
:1008B00080EA610100E04910601CC4B2082CF2DB40
:1008C000581CC3B2AB42EADB081200EB012081B234
:1008D0000846DCE710B5024800F042FD10BD0000FC
:1008E0005406002010B5024800F03AFD10BD00008B
:1008F000F405002010B5024800F032FD10BD0000E4
:10090000F803002010B5024800F02AFD10BD0000D9
:10091000B804002010B5024800F022FD10BD000010
:10092000580400200146087810381823B0FBF3F271
:100930000848805CC865032A05D908686FF3090078
:10094000001D886503E008686FF309008865886DFD
:1009500070470000BCA00008014600208A6A8B692D
:10096000CBB932B1012A0DD0022A03D0032A10D10B
:100970000EE000BFCB6A03F08073B3F1807F00D13B
:10098000012007E0CB6AB3F1C07F00D1012001E074
:1009900000E000BF34E08B69B3F5005F1AD132B1DB
:1009A000012A07D0022A03D0032A11D10AE000BF8E
:1009B00001200EE0CB6A03F08073B3F1807F00D199
:1009C000012006E0CB6AB3F1C07F00D1012000E036
:1009D00000BF15E032B1012A05D0022A04D0032A53
:1009E0000CD103E000BF00BF012008E0CB6A03F098
:1009F0008073B3F1807F00D1012000E000BF00BF11
:100A0000704730B50468246824F4802405682C609D
:100A1000046863608468402C04D10468A2600468A0
:100A2000E16003E00468A1600468E26030BD7047E3
:100A300072B600BFFEE7000038B502460020009005
:100A400000BF92F83C00012801D1022038BD0120EE
:100A500082F83C0000BF0868092816D91068C068F1
:100A60000C780A3C04EB44050724AC40A04314680E
:100A7000E0600C780A3C04EB44048868A0401468E9
:100A8000E46820431468E06013E0106800690C78A3
:100A900004EB44050724AC40A043146820610C78A3
:100AA00004EB44048868A040146824692043146857
:100AB00020614868072817D21068406B0C79641EC3
:100AC00004EB84051F24AC40A043146860630888CD
:100AD00080B20C79641E04EB8404A0401468646B3B
:100AE00020431468606331E048680D2817D210680D
:100AF000006B0C79E41F04EB84051F24AC40A04379
:100B000014682063088880B20C79E41F04EB840425
:100B1000A0401468246B20431468206316E010681A
:100B2000C06A0C790D3C04EB84051F24AC40A04343
:100B30001468E062088880B20C790D3C04EB8404F0
:100B4000A0401468E46A20431468E062194B1A4C10
:100B50001068A04206D10868122803D1586840F4F2
:100B600080005860144C1068A0421CD108681028FE
:100B700002D00868112816D1586840F40000586067
:100B8000086810280FD10D4800680D4CB0FBF4F038
:100B900000EB80004000009002E00098401E0090B2
:100BA00000980028F9D100BF002082F83C0000BF67
:100BB00000BF4BE700230140002001402C00002033
:100BC00040420F00704770477047000070B5044600
:100BD00000250CB9012070BD1549A06A884200D0DB
:100BE00000BF206C30B9204600F024F8002060647B
:100BF00084F83C00206C00F0100088B9206C20F4D0
:100C0000885040F0020020642046FFF789FD002054
:100C10006064206C20F0020040F00100206400E0DD
:100C2000012500BF002084F83C0000BF2846D2E721
:100C30000100000F10B586B00446142101A8FFF78B
:100C40006BFB86492068884263D100BF002000907A
:100C50008348006840F48070814908600846006855
:100C600000F48070009000BF00BF00BF0020009023
:100C70007B481438006840F0040079491439086052
:100C80000846006800F00400009000BF00BF00BFED
:100C9000002000900846006840F001000860084607
:100CA000006800F00100009000BF00BF3F200190ED
:100CB000032002900020039001A96A4800F030FD53
:100CC000CF200190032002900020039001A96648E4
:100CD00000F026FD65486649086000204860002154
:100CE00063488160C1604FF48061016189004161A6
:100CF000890081618911C16100210162416200F0B6
:100D00004FFC08B1FFF794FE00BF5948A06384630D
:100D1000A1E05849206888424BD100BF00200090D4
:100D20004F48006840F400704D490860084600686C
:100D300000F40070009000BF00BF00BF00200090D2
:100D400047481438006840F00200454914390860EB
:100D50000846006800F00200009000BF00BF0320BA
:100D6000019002900020039001A9434800F0D8FCB4
:100D70003E483030414908604FF000704860002123
:100D80003E488160C1604FF480610161890041612A
:100D9000890081618911C16100210162416200F015
:100DA000FFFB08B1FFF744FE00BF3448A063846333
:100DB00051E03349206888424DD100BF00200090A7
:100DC0002748006840F480602549086008460068AC
:100DD00000F48060009000BF00BF00BF00200090C2
:100DE0001F481438006840F020001D49143908607D
:100DF0000846006800F02000009000BF00BF4FF4DC
:100E0000FF600190032002900020039001A91D487B
:100E100000F086FC154818301B4908604FF08060D0
:100E20004860002118488160C1604FF48061016111
:100E300089004161890081618911C16100210162DC
:100E4000416200F0ADFB08B1FFF7F2FD00BF0E48B4
:100E5000A063846300BF06B010BD00000020014005
:100E60004438024000080240000002401064024082
:100E7000F803002000210140000402405804002033
:100E80000022014000140240B8040020F8B50446D6
:100E90000D4616460020009000BF94F83C00012843
:100EA00001D10220F8BD012084F83C0000BF206879
:100EB000806800F00100A0B92068806840F001005F
:100EC00021688860554800685549B0FBF1F000EB97
:100ED0004000009002E00098401E0090009800281A
:100EE000F9D12068806800F48070B0F5807F05D16A
:100EF0002068806820F4807021688860206880689D
:100F000000F0010000287ED0206C40F2016188438F
:100F100040F4807020642068406800F4806028B14C
:100F2000206C20F4005040F480502064206C00F4C9
:100F30008050B0F5805F04D1606C20F006006064E2
:100F400001E00020606400BF002084F83C0000BF86
:100F5000344F3548A16BC8633448A16B08643448EA
:100F6000A16BC8646FF022002168086020684068A7
:100F700040F08060216848602068806840F480709C
:100F800021688860226802F14C0133462A46A06B32
:100F900000F07CFB786800F01F0018BB2549206832
:100FA000884213D024492068884204D1381D006843
:100FB00000F01F0050B12149206888422BD1194808
:100FC000001D006800F01F00102824D220688068EF
:100FD00000F04050F8B92068806840F080402168F7
:100FE000886018E013492068884214D1206880681E
:100FF00000F0405078B92068806840F08040216857
:10100000886008E0FFE7206C40F010002064606C0E
:1010100040F001006064002044E700002C00002044
:1010200040420F0000230140790600081107000824
:10103000F706000800200140002101400022014085
:101040007047F0B5034600BF5879012801D102204E
:10105000F0BD0120587100BF0220187118680468A3
:1010600002F0100640F6FE70B0408443D1E900065D
:1010700040EA060502F0100005FA00F00443186883
:1010800004601868006802F01007C026BE40B04334
:101090001E6830600120187100BF0020587100BF29
:1010A00000BFD5E7704710B504462068006800F41B
:1010B0000050B0F5005F19D12068406B00F400507B
:1010C000B0F5005F12D104202071206940F00100CA
:1010D00020614FF40050216848632068006820F4C4
:1010E0008050216808602046FFF7DCFF2068006818
:1010F00000F00050B0F1005F19D12068406B00F0A3
:101100000050B0F1005F12D104202071206940F03E
:10111000020020614FF00050216848632068006899
:1011200020F08050216808602046FFF789FF10BD3D
:1011300010B504460CB9012010BD207920B900205B
:101140006071204600F008F8022020710020206124
:10115000012020710020EFE710B586B0044614216D
:1011600001A8FFF7D9F81D492068884233D100BF94
:10117000002000901A48006840F0005018490860AC
:101180000846006800F00050009000BF00BF00BF9C
:101190000020009012481038006840F0010010490B
:1011A000103908600846006800F00100009000BF98
:1011B00000BF30200190032002900020039001A97D
:1011C000084800F0ADFA00220F21362000F07EFC26
:1011D000362000F06BFC06B010BD0000007400402B
:1011E000403802400000024038B50446002000901C
:1011F0002068009029B902F10800009D2844009061
:1012000004E002F11400009D28440090009803605F
:10121000002038BD10B5024600BF5079012801D129
:10122000022010BD0120507100BF02201071106813
:10123000006801F010040123A340184313681860EC
:1012400061B91068006800F03C003C2816D11068B5
:10125000406840F00100136858600FE010680068B3
:1012600000F4701301F010043C20A040834205D12B
:101270001068406840F00200136858600120107147
:1012800000BF0020507100BF00BFCAE770B5044620
:10129000A56D00F057FB064694F83500022808D0EB
:1012A0008020606500BF002084F8340000BF01206A
:1012B00070BD2068006820F0160021680860206872
:1012C000406920F0800021684861206C08B9A06C5A
:1012D00028B12068006820F00800216808602068B4
:1012E000006820F001002168086010E000F02AFB8F
:1012F000801B05280BD920206065032084F8350069
:1013000000BF002084F8340000BF0320D0E720682D
:10131000006800F001000028E8D194F85C103F203C
:101320008840A860012084F8350000BF002084F8C0
:10133000340000BF00BFBBE7014691F8350002282A
:1013400003D08020486501207047052081F83500D2
:101350000868006820F001000A6810600020F3E7C8
:10136000F8B50446002000908C4800684FF41651F0
:10137000B0FBF1F7A56D2E6894F85C10082088404A
:10138000304098B12068006800F0040070B1206817
:10139000006820F004002168086094F85C100820C0
:1013A0008840A860606D40F00100606594F85C10B2
:1013B00001208840304068B12068406900F080001A
:1013C00040B194F85C1001208840A860606D40F046
:1013D0000200606594F85C1004208840304068B1D9
:1013E0002068006800F0020040B194F85C1004200E
:1013F0008840A860606D40F00400606594F85C105F
:1014000010208840304078B32068006800F0080061
:1014100050B394F85C1010208840A86020680068E1
:1014200000F4802080B12068006800F4002028B912
:10143000206CC8B12046216C884715E0A06C98B19B
:101440002046A16C88470FE02068006800F4807097
:1014500028B92068006820F0080021680860206C26
:1014600010B12046216C884794F85C1020208840F9
:101470003040002865D02068006800F01000002887
:101480005FD094F85C1020208840A86094F8350064
:10149000052828D12068006820F01600216808601F
:1014A0002068406920F0800021684861206C08B9FC
:1014B000A06C28B12068006820F00800216808604E
:1014C00094F85C103F208840A860012084F8350023
:1014D00000BF002084F8340000BF206D10B120460A
:1014E000216D8847F8BD2068006800F4802080B135
:1014F0002068006800F4002028B9606C10B1204614
:10150000616C88471DE0E06BD8B12046E16B8847ED
:1015100017E02068006800F4807068B920680068EF
:1015200020F0100021680860012084F8350000BF19
:10153000002084F8340000BFE06B10B12046E16B5E
:101540008847606D38B3606D00F00100F0B1052090
:1015500084F835002068006820F0010021680860E8
:1015600000BF0098401C0090B84200D905E02068F8
:10157000006800F001000028F3D100BF012084F8CA
:10158000350000BF002084F8340000BFE06C10B1CB
:101590002046E16C884700BFA4E700002C00002033
:1015A0002DE9F0410446002500F0CCF9074614B9B6
:1015B0000120BDE8F081606A00B100BF022084F81C
:1015C000350000BF002084F8340000BF20680068A8
:1015D00020F00100216808600AE000F0B3F9C01BA8
:1015E000052805D920206065032084F83500E0E750
:1015F0002068006800F001000028EED1206805682E
:1016000021480540D4E901010843E1680843216904
:10161000084361690843A1690843E1690843216AF5
:1016200008430543606A042803D1D4E90B01084349
:101630000543206805602068456925F00705606A54
:101640000543606A04280DD1A06A0543E06A48B1E9
:101650002046FFF781F928B140206065012084F819
:101660003500A6E7206845612046FFF75BF906468E
:1016700094F85C103F208840B06000206065012035
:1016800084F83500002094E73F8010F02DE9F04702
:1016900004460D4616461F464FF00008D4F85890F1
:1016A00000BF94F83400012802D10220BDE8F08781
:1016B000012084F8340000BF94F83500012825D1BA
:1016C000022084F83500002060653B4632462946FA
:1016D0002046FFF796F994F85C103F208840C9F83F
:1016E00008002068006840F0160021680860206C3F
:1016F00028B12068006840F0080021680860206870
:10170000006840F001002168086006E000BF00208A
:1017100084F8340000BF4FF002084046C6E70000DE
:10172000F8B502460B460025002400200021D6E033
:10173000012606FA01F51E6806EA0504AC4274D1DA
:101740001E7906F00306012E04D01E7906F003066A
:10175000022E13D190684F000326BE40B0434F00C5
:10176000DE68BE4030439060506801268E40B04332
:101770001E79C6F300168E40304350601E7906F085
:101780000306032E09D0D0684F000326BE40B043A5
:101790004F009E68BE403043D0601E7906F00306BD
:1017A000022E13D1CF0802F1200656F827004E076B
:1017B000F70E0F26BE40B0434F07FF0E1E69BE4016
:1017C0003043CF0802F1200646F8270010684F008A
:1017D0000326BE40B0431E7906F003064F00BE400C
:1017E000304310605E6806F44036002E76D000BFAD
:1017F000002600963C4E366846F480463A4F3E60DE
:101800003E46366806F48046009600BF00BF374E5D
:101810008F0856F827008E07370F0F26BE40B043BB
:10182000334EB24202D1002624E057E0314EB2429C
:1018300001D101261EE0304EB24201D1022619E04C
:101840002E4EB24201D1032614E02D4EB24201D1F8
:1018500004260FE02B4EB24201D105260AE02A4EA3
:10186000B24201D1062605E0284EB24201D1072638
:1018700000E008268F073F0FBE4030431B4E8F0805
:1018800046F82700224E3068A0435E6806F48016B2
:1018900006B120431E4E3060361D3068A0435E689E
:1018A00006F4001606B12043194E361D3060184E5E
:1018B000361F3068A0435E6806F4003606B1204348
:1018C000134E361F3060361F3068A0435E6806F442
:1018D000803606B120430E4E083E3060491C102968
:1018E000FFF426AFF8BD000044380240083801403C
:1018F000000002400004024000080240000C0240C8
:10190000001002400014024000180240001C024077
:10191000083C0140024613690B400BB1012000E076
:101920000020704710B5426921EA020302EA01046F
:1019300043EA0443836110BD0AB1816101E00B04F5
:101940008361704701480068704700002000002054
:101950000348006803490978084401490860704752
:10196000200000202800002010B50D48006840F439
:1019700000700B4908600846006840F48060086009
:101980000846006840F480700860032000F0DCF82E
:101990000F2000F007F800F05FF8002010BD0000F5
:1019A000003C02402DE9F04188B004460027B846CB
:1019B00000BF002001902348006840F0100021493A
:1019C00008600846006800F01000019000BF00BFEA
:1019D00002A903A800F08EF9069F1FB900F0B2F922
:1019E000054602E000F0AEF945001748B5FBF0F0FF
:1019F000A0F1010815481649086040F2E731144883
:101A0000C160C0F80480002101618160816100F043
:101A1000C9FF064696B90E4801F05AF806466EB957
:101A2000362000F043F8102C07D200222146362041
:101A300000F04CF80748046000E00126304608B08A
:101A4000BDE8F0814038024040420F0000100040E5
:101A5000300900202400002008B500BF00200090BD
:101A60001148006840F480400F490860084600684B
:101A700000F48040009000BF00BF00BF0020009035
:101A8000081F006840F08050091F08600846006881
:101A900000F08050009000BF00BF00220F21901E78
:101AA00000F014F808BD0000443802400146084622
:101AB000002809DB00F01F0301229A4043099B0024
:101AC00003F1E023C3F8002100BF70472DE9F05F68
:101AD00080460D461646002703F028FF0746394684
:101AE0002A46334601F00700C0F1070ABAF1040F95
:101AF00002D94FF0040A01E0C0F1070AD14600F113
:101B0000040ABAF1070F02D24FF0000A01E0A0F177
:101B1000030AD4464FF0010A0AFA09FAAAF1010AA7
:101B20000AEA020A0AFA0CFA4FF0010B0BFA0CFB54
:101B3000ABF1010B0BEA030B4AEA0B0421464046CA
:101B400003F0FCFEBDE8F09F00BF00F00702064B6B
:101B500019684FF6FF031940044B0B4343EA022177
:101B6000014B196000BF70470CED00E00000FA0562
:101B700070B504460D460CB9012070BD5848006888
:101B800000F00700A84209D255490D7008460068C8
:101B900000F00700A84201D00120EEE7207800F015
:101BA000020002281DD1207800F00400042805D18D
:101BB0004C48006840F4E0504A490860207800F042
:101BC0000800082805D14748006840F460404549AE
:101BD00008604448006820F0F000A16808434149CB
:101BE0000860207800F00100A8B36068012807D1E0
:101BF0003C4808380068C0F34040B8B90120BCE751
:101C00006068022802D06068032807D13548083888
:101C10000068C0F3406048B90120AEE73148083899
:101C20000068C0F3400008B90120A6E72D4800680D
:101C300020F00300616808432A490860FFF782FE2C
:101C4000064609E0FFF77EFE801B41F2883188429C
:101C500002D9032091E707E02248006800F00C0059
:101C60006168B0EB810FEDD11D48006800F00700FE
:101C7000A84209D91A490D700846006800F007000B
:101C8000A84201D0012078E7207800F00400042861
:101C900007D11448006820F4E050E1680843114976
:101CA0000860207800F00800082808D10D48006876
:101CB00020F46040216940EAC1000A49086000F050
:101CC00061F808490968C1F30311074A515CC8402B
:101CD0000649086006480068FFF764FE00204CE7EC
:101CE000003C024008380240C4A000082C0000203C
:101CF000240000200F2202600D4A126802F0030245
:101D000042600B4A126802F0F0028260084A1268D0
:101D100002F4E052C260064A126802F46042D2083D
:101D20000261044A126802F007020A60704700006C
:101D300008380240003C024001480068704700003B
:101D40002C00002000B5FFF7F7FF04490968C1F334
:101D50008221034A515CC84000BD0000083802409F
:101D6000D4A0000800B5FFF7E7FF04490968C1F3F4
:101D70004231034A515CC84000BD000008380240AF
:101D8000D4A000082DE9F047002400250026A14634
:101D90002548006800F00C0020B1042805D0082870
:101DA0003AD105E0DFF8849039E0DFF8849036E03E
:101DB0001D48001F006800F03F041B48001F00681A
:101DC00000F4800078B11A481749091F0968C1F367
:101DD0008811A0FB01700146224600233846FEF719
:101DE00051FA05460EE011480F49091F0968C1F371
:101DF0008811A0FB01700146224600233846FEF7F9
:101E000041FA05460848001F0068C0F30140401C25
:101E10004600B5FBF6F902E0DFF8109000BF00BF06
:101E20004846BDE8F0870000083802400024F4006E
:101E300040787D01F8B504460CB90120F8BD207842
:101E400000F00100002874D0F948006800F00C0090
:101E500004280DD0F648006800F00C00082813D1C3
:101E6000F348001F006800F48000B0F5800F0BD12C
:101E7000EF4808380068C0F34040002859D0606837
:101E8000002856D10120D9E700BF6068B0F5803F37
:101E900008D1E7480838006840F48030E449083940
:101EA00008601EE06068B0F5A02F0DD1E04808384A
:101EB000006840F48020DE49083908600846006860
:101EC00040F4803008600CE0D9480838006820F4FD
:101ED0008030D749083908600846006820F480201F
:101EE000086000BF606890B1FFF72CFD054606E072
:101EF000FFF728FD401B642801D903209EE7CC484A
:101F000008380068C0F340400028F1D011E0FFF726
:101F100019FD054606E0FFF715FD401B642801D9B1
:101F200003208BE7C24808380068C0F3404000280F
:101F3000F1D1207800F0020002285FD1BC4800688F
:101F400000F00C0058B1BA48006800F00C000828F6
:101F50001CD1B748001F006800F48000B0B9B44835
:101F600008380068C0F3400020B1E068012801D0C3
:101F7000012063E7AE480838006820F0F8002169C6
:101F800040EAC100AA490839086037E0E06800B3B8
:101F90000120A8490860FFF7D5FC054606E0FFF7D9
:101FA000D1FC401B022801D9032047E7A04808388C
:101FB0000068C0F340000028F1D09D480838006850
:101FC00020F0F800216940EAC10099490839086009
:101FD00014E0002097490860FFF7B4FC054606E0CE
:101FE000FFF7B0FC401B022801D9032026E79048E8
:101FF00008380068C0F340000028F1D1207800F0D4
:10200000080008282CD16069A8B101208A4908601D
:10201000FFF798FC054606E0FFF794FC401B0228FA
:1020200001D903200AE782486C300068C0F3400001
:102030000028F1D014E000207F490860FFF782FCFF
:10204000054606E0FFF77EFC401B022801D903206D
:10205000F4E677486C300068C0F340000028F1D106
:10206000207800F00400042870D100277048383030
:10207000006800F0805090B900BF002000906C48CC
:102080003830006840F080506949383108600846AF
:10209000006800F08050009000BF00BF0127674833
:1020A000006800F48070B0B96448006840F4807043
:1020B00062490860FFF746FC054606E0FFF742FC70
:1020C000401B022801D90320B8E65C48006800F4F0
:1020D00080700028F2D000BFA068012808D15448C1
:1020E0006830006840F001005149683108601DE027
:1020F000A06805280DD14E486830006840F0040003
:102100004B49683108600846006840F001000860EB
:102110000CE047486830006820F00100444968310D
:1021200008600846006820F00400086000BFA0684E
:10213000A8B1FFF707FC054609E0FFF703FC401BC9
:1021400041F28831884202D9032077E626E03848F8
:1021500068300068C0F340000028EED013E0FFF7BD
:10216000F1FB054608E0FFF7EDFB401B41F288312B
:10217000884201D9032061E62D4868300068C0F329
:1021800040000028EFD1012F07D1294838300068DE
:1021900020F0805026493831086000BFA06900282F
:1021A00045D02348006800F00C0008285DD0A069E5
:1021B000022845D100201F490866FFF7C3FB0546EA
:1021C00006E0FFF7BFFB401B022801D9032035E6DC
:1021D000174808380068C0F340600028F1D1D4E9FE
:1021E00007010843616A40EA81110122A06AC2EB3B
:1021F000500041EA00412C20005D41EA00600C499A
:10220000091F086001200B490866FFF79BFB054684
:1022100006E0FFF797FB401B022801D903200DE6DB
:10222000034808380068C0F340600028F1D049E056
:102230000838024000004742800E474200700040CC
:10224000002021490866FFF77DFB054606E0FFF701
:1022500079FB401B022801D90320EFE51B480068E9
:10226000C0F340600028F2D12CE0A069012800D121
:10227000E4E51648001D0668A069012820D006F490
:102280008001E06981421BD106F03F01206A814252
:1022900016D147F6C0703040616AB0EB811F0FD194
:1022A00006F440310122A06AC2EB5000B1EB004FAE
:1022B00006D106F070612C20005DB1EB006F01D0FB
:1022C0000120BBE50020B9E500004742003802408C
:1022D00010B504460CB9012010BD606A38B96068B9
:1022E000B0F5827F00D105E00021E16102E000212C
:1022F000216161610021A16294F8510028B9002098
:1023000084F85000204600F047F8022084F851007D
:102310002068006820F0400021680860A08800F470
:102320008270218901F404410843A18901F400610C
:102330000843217C01F002010843217D01F00101E5
:102340000843218B01F400710843217F01F038011B
:1023500008432021095D01F080010843218D01F42B
:1023600000510843216808600421A06901EA104077
:1023700094F8241001F01001084321684860206897
:10238000C06920F400602168C861002060650120F8
:1023900084F8510000209FE710B586B00446142150
:1023A00001A8FDF7B9FF54492068884230D100BF29
:1023B000002000905148006840F480504F49086068
:1023C0000846006800F48050009000BF00BF00BFC6
:1023D0000020009049481438006840F00200474946
:1023E000143908600846006800F00200009000BF41
:1023F00000BF2820019002200290002003900320BB
:1024000004900520059001A93D48FFF789F970E087
:102410003C49206888426CD100BF002000903748BA
:10242000001F006840F480403449091F08600846D6
:10243000006800F48040009000BF00BF00BF002093
:1024400000902E481438006840F002002B491439DF
:1024500008600846006800F00200009000BF00BF5E
:102460004FF460400190022002900020039003206E
:1024700004900520059001A92148FFF751F9224851
:1024800022490860002048604021204881600021E6
:10249000C1604FF480610161002141618161C161CE
:1024A00001624162FFF77CF808B1FEF7C1FA00BF94
:1024B0001648A064846300BF1348183814490860A4
:1024C00000204860002112488160C1604FF48061A3
:1024D0000161002141618161C16101624162FFF7D7
:1024E0005FF808B1FEF7A4FA00BF0948E06484630E
:1024F00000BF06B010BD000000300140443802406B
:10250000000402400038004070600240F4050020E2
:10251000540600202DE9F84F0446884616461D460D
:102520004FF0000A00BF94F85000012802D10220A9
:10253000BDE8F88F012084F8500000BFFFF702FAD1
:102540000746B14694F85100012802D04FF0020A24
:10255000ADE0B8F1000F00D016B94FF0010AA6E0C7
:10256000032084F8510000206065C4F83080A686FE
:10257000E686A063A087E08760642064A068B0F569
:10258000004F0BD12068006820F0400021680860EF
:102590002068006840F48040216808602068006876
:1025A00000F04000402805D02068006840F040005E
:1025B00021680860E068B0F5006F2FD1606810B145
:1025C000B9F1010F09D1206B00882168C860206B28
:1025D000801C2063E08E401EE0861BE0206880683F
:1025E00000F0020002280AD1206B00882168C86030
:1025F000206B801C2063E08E401EE0860AE0FFF71F
:10260000A1F9C01BA84201D3681C00B915B94FF04D
:10261000030A4CE0E08E0028E0D12EE0606810B1A3
:10262000B9F1010F09D1206B007821680873206B84
:10263000401C2063E08E401EE0861BE0206880681E
:1026400000F0020002280AD1206B0078216808738C
:10265000206B401C2063E08E401EE0860AE0FFF7FE
:1026600071F9C01BA84201D3681C00B915B94FF01D
:10267000030A1CE0E08E0028E0D13A4629462046B5
:1026800002F06EFB08B120206065A06850B900BF61
:10269000002000902068C06800902068806800904A
:1026A00000BF00BF606D08B14FF0010A00BF0120FC
:1026B00084F8510000BF002084F8500000BF50464D
:1026C00036E72DE9FF5F0446884691461D460E9E7B
:1026D000012002900020019000BF94F850000128D2
:1026E00003D1022004B0BDE8F09F012084F850001F
:1026F00000BFFFF727F9074694F851B060680390D0
:10270000AA46BBF1010F0BD00398B0F5827F04D12C
:10271000A06810B9BBF1040F02D002200190DBE0E9
:10272000B8F1000F03D0B9F1000F00D015B90120A6
:102730000190D1E094F85100042802D0052084F8DB
:10274000510000206065C4F83890E587A587C4F87B
:102750003080E586A586206460642068006800F00B
:102760004000402805D02068006840F04000216803
:102770000860E068B0F5006F4AD1606810B1BAF146
:10278000010F09D1206B00882168C860206B801C74
:102790002063E08E401EE08633E02068806800F011
:1027A0000200022810D1E08E70B1029801280BD1EE
:1027B000206B00882168C860206B801C2063E08E3D
:1027C000401EE086002002902068806800F0010032
:1027D00068B1E08F58B12068C068A16B0880A06B19
:1027E000801CA063E08F401EE08701200290FFF76D
:1027F000A9F8C01BB04204D3701C10B10320019093
:102800006AE0E08E0028C8D1E08F0028C5D14AE0F8
:10281000606810B1BAF1010F09D1206B007821680E
:102820000873206B401C2063E08E401EE08634E07D
:102830002068806800F00200022810D1E08E70B19C
:10284000029801280BD1206B007821680873206B57
:10285000401C2063E08E401EE0860020029020682D
:10286000806800F0010068B1E08F58B12068C0684E
:10287000A16B0870A06B401CA063E08F401EE08736
:1028800001200290FFF75EF8C01BB04201D3701C1C
:1028900000B916B9032001901EE0E08E0028C7D1D0
:1028A000E08F0028C4D13A463146204602F058FA5B
:1028B00020B101200190202060650DE0A06850B992
:1028C00000BF002000902068C068009020688068E9
:1028D000009000BF00BF00BF012084F8510000BF7E
:1028E000002084F8500000BF0198FBE67047704755
:1028F00030B502460B4600BF92F83C00012801D1DA
:10290000022030BD012082F83C0000BF022082F886
:102910003D00106844681068816824F070041868ED
:10292000044310684460184D1068A8421BD010681A
:10293000B0F1804F17D0154D1068A84213D0144D38
:102940001068A8420FD0134D1068A8420BD0124D4A
:102950001068A84207D0114D1068A84203D0104D4E
:102960001068A84205D121F0800158680143106821
:102970008160012082F83D0000BF002082F83C0009
:1029800000BF00BFBDE700000000014000040040A0
:1029900000080040000C00400004014000400140DD
:1029A0000018004010B504460CB9012010BD94F881
:1029B0003D0028B9002084F83C00204600F026F8AD
:1029C000022084F83D00211D206802F039FB01201F
:1029D00084F8460000BF84F83E0001213F200155E5
:1029E000402001554120015500BF00BF012084F85F
:1029F000420043200155442001554520015500BFA8
:102A0000012084F83D000020D0E7000010B586B01A
:102A10000446142101A8FDF77FFC2949206888425B
:102A200037D100BF002000902648006840F40030F5
:102A3000244908600846006800F40030009000BF98
:102A400000BF00BF002000901E481438006840F00E
:102A500002001C49143908600846006800F00200B2
:102A6000009000BF00BF8815019012200290002046
:102A7000039004900320059001A91348FEF750FE2F
:102A8000002205211920FFF721F81920FFF70EF881
:102A900013E00E49206888420FD100BF002000904B
:102AA0000848006840F4802006490860084600682D
:102AB00000F48020009000BF00BF06B010BD0000F1
:102AC00000440140443802400004024000480140F4
:102AD000014691F83D00012801D0012070470220F5
:102AE00081F83D000868C06840F001000B68D860BC
:102AF0001A4B086898421BD00868B0F1804F17D075
:102B0000174B0868984213D0164B086898420FD0AC
:102B1000154B086898420BD0144B0868984207D0B0
:102B2000134B0868984203D0124B086898420CD1A6
:102B30000868806800F00702062A0CD00868006860
:102B400040F001000B68186005E00868006840F07C
:102B500001000B6818600020C0E700000000014081
:102B60000004004000080040000C00400004014048
:102B7000004001400018004001460868C06820F08D
:102B800001000A68D06000BF0868006A41F21112B3
:102B9000104050B90868006A9210104028B90868BF
:102BA000006820F001000A68106000BF012081F871
:102BB0003D00002070472DE9F04104460D4614B950
:102BC0000120BDE8F08194F83D0028B9002084F888
:102BD0003C00204600F054F8022084F83D002068B4
:102BE000806844F20701884321688860211D2068BD
:102BF00002F026FA2068D0F80880206886692068EC
:102C0000076A286840EA080840F203308643A96949
:102C1000A86840EA0120064340F60C4086434FF284
:102C2000F0008643E969E86840EA01200643286924
:102C30000001296A40EA0130064327F0220727F005
:102C400088076969686840EA011007432068C0F88E
:102C500008802068866120680762012084F84600A9
:102C600084F83E0001213F200155012084F84200F4
:102C700043200155012084F83D000020A1E7000019
:102C800010B586B00446142101A8FDF745FB3E4966
:102C90002068884240D100BF002000903B48006877
:102CA00040F00100394908600846006800F0010062
:102CB000009000BF00BF00BF0020009033481438D0
:102CC000006840F001003149143908600846006886
:102CD00000F00100009000BF00BF4FF44070019071
:102CE000022002900020039004900120059001A989
:102CF0002748FEF715FD002205211820FEF7E6FE05
:102D00001820FEF7D3FE002205211920FEF7DEFE73
:102D10001920FEF7CBFE34E01E492068884230D1EE
:102D200000BF002000901948001F006840F002001A
:102D30001649091F08600846006800F0020000906C
:102D400000BF00BF00BF002000901048143800688A
:102D500040F004000D49143908600846006800F08E
:102D60000400009000BF00BFC0200190022002902C
:102D70000020039004900220059001A90648FEF768
:102D8000CFFC06B010BD00000000014044380240F6
:102D90000000024000040040000802402DE9F0431A
:102DA00004460D4694F83E603F20075D94F842804B
:102DB000432010F804906DB9012E02D1B8F1010F33
:102DC00002D00120BDE8F083022084F83E0084F8A0
:102DD000420025E0042D0CD1012F02D1B9F1010FE1
:102DE00001D00120EEE702213F200155432001558B
:102DF00016E0012E07D1012F05D1B8F1010F02D144
:102E0000B9F1010F01D00120DCE7022084F83E0077
:102E100002213F200155022084F842004320015541
:102E200015B1042D0CD105E001220021206802F02B
:102E300073F910E001220421206802F06DF90AE024
:102E400001220021206802F067F901220421206894
:102E500002F062F900BF00BF2068006840F0010086
:102E6000216808600020ADE72DE9F04F2DED048BBF
:102E700085B08246BAF1000F04D105B0BDEC048BD9
:102E8000BDE8F08F5748824503D104200490564C8A
:102E900005E05648824502D100200490544C254656
:102EA00004F1040804F108000390061D04F1100960
:102EB0000C300290071D04F11C0B0C3001904FF4F4
:102EC000FA7101980160386818B93868401C386098
:102ED00001E0002038603868012806D10020DAF8C7
:102EE00000104862CBF800007AE03868002877D1FB
:102EF0005046049900F074FE28602868DBF8001042
:102F0000C1EB0141084403990860039890ED000A61
:102F1000B8EE400ADFED370A80EE801A86ED001A1F
:102F200096ED000ADFED340AB4EEE00AF1EE10FA95
:102F300003DD9FED310A86ED000A96ED000AD9ED1A
:102F4000000A30EE600A10EE101A0846FDF76EFA1D
:102F500041EC190BB0EE490AF0EE690A02F002FDED
:102F6000B0EE408AF0EE608A9FED240B53EC102BFC
:102F700051EC180BFDF786FA14D299ED000A86ED94
:102F8000000AD8F80000401CC8F80000D8F800007B
:102F900005281CD996ED000A89ED000A0020C8F822
:102FA000000014E00020C8F8000099ED000ADFEDF1
:102FB000150A20EE200AD6ED000A9FED131A00EE46
:102FC000810A86ED000A96ED000A89ED000A96ED69
:102FD000000ADFED0E0A20EE200A029880ED000ABA
:102FE00000BF4AE78C07002018770020D407002094
:102FF000F47600200024744900008844000000009A
:1030000000004940CDCC4C3FCDCC4C3E000070423E
:103010002DE9F04104460D461646002700BF94F8FE
:103020003C00012802D10220BDE8F081012084F893
:103030003C0000BF96B9EB68D5E90012206802F0A9
:1030400059F92068806920F00C00216888612068A7
:103050008069A96808432168886141E0042E13D182
:10306000EB68D5E90012206802F08CF920688069CD
:1030700020F440602168886120688069A96840EA7E
:103080000120216888612BE0082E12D1EB68D5E978
:103090000012206802F093F92068C06920F00C004B
:1030A0002168C8612068C069A96808432168C861AF
:1030B00016E00C2E13D1EB68D5E90012206802F05F
:1030C0009AF92068C06920F440602168C8612068CE
:1030D000C069A96840EA01202168C86100E00127B1
:1030E00000BF002084F83C0000BF38469CE710B5C4
:1030F00004460CB9012010BD94F83D0028B9002009
:1031000084F83C00204600F025F8022084F83D00B9
:10311000211D206801F094FF012084F8460000BFC3
:1031200084F83E0001213F200155402001554120F7
:10313000015500BF00BF012084F842004320015523
:10314000442001554520015500BF012084F83D0071
:103150000020D0E710B586B00446142101A8FDF781
:10316000DBF81E492068884236D100BF002000905D
:103170001B48006840F48030194908600846006820
:1031800000F48030009000BF00BF00BF002000901E
:1031900013481438006840F01000114914390860D1
:1031A0000846006800F01000009000BF00BF4020FB
:1031B00001901220029000200390049003200590BB
:1031C00001A90848FEF7ACFA002205211820FEF7F5
:1031D0007DFC1820FEF76AFC06B010BD00400140DF
:1031E00044380240001002402DE9F04304460D46E9
:1031F000002615B994F83E000BE0042D02D13F20C3
:10320000005D06E0082D02D14020005D01E0412074
:10321000005D804615B994F842000BE0042D02D100
:103220004320005D06E0082D02D14420005D01E04E
:103230004520005D8146B8F1010F02D1B9F1010FBF
:1032400002D00120BDE8F0831DB9022084F83E00C1
:103250000EE0042D03D102213F20015508E0082D86
:1032600003D102214020015502E0022141200155F5
:103270001DB9022084F842000EE0042D03D1022182
:103280004320015508E0082D03D1022144200155B7
:1032900002E002214520015535B1042D0BD0082D47
:1032A00010D00C2D1CD114E02068C06840F0020042
:1032B0002168C86016E02068C06840F004002168FA
:1032C000C8600FE02068C06840F008002168C8604E
:1032D00008E02068C06840F010002168C86001E084
:1032E000012600BF00BF86BB01222946206801F0ED
:1032F00013FF1A49206888421BD02068B0F1804F24
:1033000017D017492068884213D016492068884290
:103310000FD01549206888420BD014492068884294
:1033200007D013492068884203D012492068884298
:103330000CD12068806800F00707062F0CD02068A9
:10334000006840F001002168086005E0206800681E
:1033500040F0010021680860304673E7000001403A
:103360000004004000080040000C00400004014040
:10337000004001400018004010B504462068006974
:10338000C0F34000D8B12068C068C0F34000B0B1BD
:103390006FF00200216808610120207720688069B1
:1033A00000F0030018B12046FFF75EFD05E020465F
:1033B00000F006F9204600F0DDF9002020772068B3
:1033C0000069C0F38000D8B12068C068C0F38000F5
:1033D000B0B16FF0040021680861022020772068F6
:1033E000806900F4407018B12046FFF73DFD05E00C
:1033F000204600F0E5F8204600F0BCF900202077D8
:1034000020680069C0F3C000D8B12068C068C0F36C
:10341000C000B0B16FF00800216808610420207777
:103420002068C06900F0030018B12046FFF71CFDBA
:1034300005E0204600F0C4F8204600F09BF900208B
:10344000207720680069C0F30010D8B12068C068F8
:10345000C0F30010B0B16FF01000216808610820BF
:1034600020772068C06900F4407018B12046FFF74B
:10347000FBFC05E0204600F0A3F8204600F07AF9B6
:10348000002020772068006900F0010058B1206812
:10349000C06800F0010030B16FF0010021680861E0
:1034A000204600F071FB20680069C0F3C01058B1DD
:1034B0002068C068C0F3C01030B16FF08000216890
:1034C00008612046FFF712FA20680069C0F38010F7
:1034D00058B12068C068C0F3801030B16FF0400070
:1034E00021680861204600F094FB20680069C0F361
:1034F000401058B12068C068C0F3401030B16FF080
:103500002000216808612046FFF7F1F910BD000096
:1035100010B586B00446142101A8FCF7FDFE23492E
:10352000206888421ED100BF00200090204800681B
:1035300040F008001E4908600846006800F00800D6
:10354000009000BF00BF4FF4404001900220029065
:103550000020039004900220059001A91548FEF771
:10356000DFF820E01449206888421CD100BF002009
:1035700000900F48006840F002000D4908600846BE
:10358000006800F00200009000BF00BF48150190E5
:10359000022002900020039004900320059001A9CE
:1035A0000648FEF7BDF806B010BD00000008004058
:1035B00030380240000C0240004801400004024044
:1035C00070472DE9F04104460D461646002700BF1E
:1035D00094F83C00012802D10220BDE8F0810120CE
:1035E00084F83C0000BF36B1042E1BD0082E31D029
:1035F0000C2E5ED145E02946206801F09FFD206831
:10360000806940F00800216888612068806920F0A6
:10361000040021688861206880692969084321685D
:10362000886148E02946206801F0C0FD2068806973
:1036300040F40060216888612068806920F480601F
:103640002168886120688069296940EA0120216831
:10365000886130E02946206801F0E6FD2068C069F5
:1036600040F008002168C8612068C06920F00400AB
:103670002168C8612068C069296908432168C86158
:1036800019E02946206801F00BFE2068C06940F46B
:1036900000602168C8612068C06920F480602168EA
:1036A000C8612068C069296940EA01202168C861B1
:1036B00001E0012700BF00BF00BF002084F83C00EC
:1036C00000BF384689E710B504460CB9012010BD8B
:1036D00094F83D0028B9002084F83C00204600F012
:1036E00025F8022084F83D00211D206801F0A8FC87
:1036F000012084F8460000BF84F83E0001213F20ED
:103700000155402001554120015500BF00BF012057
:1037100084F84200432001554420015545200155BD
:1037200000BF012084F83D000020D0E738B50446F2
:103730000E492068884217D100BF002000900C4835
:10374000006840F004000A4908600846006800F07C
:103750000400009000BF00BF002205211E20FEF7DC
:10376000B5F91E20FEF7A2F938BD000000080040A0
:10377000403802407047000070B504460D4615B948
:1037800094F83E000BE0042D02D13F20005D06E0DE
:10379000082D02D14020005D01E04120005D01289C
:1037A00001D0012070BD1DB9022084F83E000EE05A
:1037B000042D03D102213F20015508E0082D03D13B
:1037C00002214020015502E0022141200155012241
:1037D0002946206801F0A0FC23492068884203D0D4
:1037E00022492068884201D1012000E0002028B150
:1037F0002068406C40F40040216848641A49206801
:1038000088421BD02068B0F1804F17D0184920683B
:10381000884213D01749206888420FD01649206883
:1038200088420BD011492068884207D0134920688C
:10383000884203D01249206888420CD120688068F1
:1038400000F00706062E0CD02068006840F001004A
:103850002168086005E02068006840F001002168E8
:10386000086000209EE700000000014000040140C5
:103870000004004000080040000C004000400140EF
:1038800000180040F0B504460D46002615B994F81E
:103890003E000BE0042D02D13F20005D06E0082D24
:1038A00002D14020005D01E04120005D012801D0EF
:1038B0000120F0BD1DB9022084F83E000EE0042D69
:1038C00003D102213F20015508E0082D03D1022138
:1038D0004020015502E002214120015535B1042D5F
:1038E0000BD0082D10D00C2D1CD114E02068C0681E
:1038F00040F002002168C86016E02068C06840F00F
:1039000004002168C8600FE02068C06840F008002B
:103910002168C86008E02068C06840F01000216895
:10392000C86001E0012600BF00BFEEBB01222946AE
:10393000206801F0F1FB24492068884203D0234924
:103940002068884201D1012000E0002028B12068D1
:10395000406C40F40040216848641B49206888425C
:103960001BD02068B0F1804F17D0194920688842D9
:1039700013D01849206888420FD017492068884220
:103980000BD012492068884207D014492068884229
:1039900003D01349206888420ED12068806800F067
:1039A0000707062F0ED000E00CE02068006840F00A
:1039B00001002168086005E02068006840F001000F
:1039C00021680860304674E70000014000040140AF
:1039D0000004004000080040000C0040004001408E
:1039E0000018004030B504460D46002229462068E4
:1039F00001F092FB23492068884203D022492068C5
:103A0000884201D1012000E0002090B100BF206871
:103A1000006A41F21111084050B92068006A89100B
:103A2000084028B92068406C20F4004021684864B0
:103A300000BF00BF2068006A41F21111084050B970
:103A40002068006A8910084028B92068006820F0C2
:103A500001002168086000BF1DB9012084F83E0004
:103A60000EE0042D03D101213F20015508E0082D6F
:103A700003D101214020015502E0012141200155DF
:103A8000002030BD000001400004014070B5044634
:103A90000D46002635B1042D0BD0082D10D00C2D6D
:103AA0001CD114E02068C06820F002002168C860C2
:103AB00016E02068C06820F004002168C8600FE0AC
:103AC0002068C06820F008002168C86008E020680D
:103AD000C06820F010002168C86001E0012600BF26
:103AE00000BF002E4AD100222946206801F014FBB5
:103AF00023492068884203D022492068884201D1A6
:103B0000012000E0002090B100BF2068006A41F26F
:103B10001111084050B92068006A8910084028B97E
:103B20002068406C20F400402168486400BF00BF5A
:103B30002068006A41F21111084050B92068006AFB
:103B40008910084028B92068006820F00100216829
:103B5000086000BF1DB9012084F83E000EE0042D6E
:103B600003D101213F20015508E0082D03D1012197
:103B70004020015502E0012141200155304670BD31
:103B8000000001400004014010B504460F492068C0
:103B9000884201D1FDF7DCFE0D492068884207D13B
:103BA0000C48006820B10B48C069401C0949C86135
:103BB00009492068884207D10848006820B10748B1
:103BC000C069401C0549C86110BD000000100040DC
:103BD000004001401877002000440140F4760020A6
:103BE0000246002031B1042907D0082908D00C2949
:103BF0000CD108E01368586B09E01368986B06E075
:103C00001368D86B03E01368186C00E000BF00BFB6
:103C100070477047704770472DE9F84F0446206899
:103C200005682068C668206847694FF00009CA46E1
:103C300005F00F09B9F1000F0AD105F0200038B1E5
:103C400006F0200020B1204601F04EFCBDE8F88FC0
:103C5000B9F1000F7CD007F0010018B906F490709C
:103C6000002875D005F0010030B106F4807018B15D
:103C7000206C40F00100206405F0040030B107F032
:103C8000010018B1206C40F00200206405F0020031
:103C900030B107F0010018B1206C40F0040020643E
:103CA00005F0080048B106F0200010B907F0010047
:103CB00018B1206C40F008002064206C002846D029
:103CC00005F0200028B106F0200010B1204601F0D8
:103CD0000BFC20684069C0F3801A206C00F00800DB
:103CE00010B9BAF1000F2DD0204601F0B7FB2068C3
:103CF000406900F04000402820D100BF00BF21688B
:103D0000143151E8001F21F040002168143141E8CE
:103D10000002002AF3D100BFA06B50B17548A16B1F
:103D20000865A06BFDF708FB88B1A06B016D8847A3
:103D30000DE02046FFF76FFF09E009E02046FFF79E
:103D40006AFF04E02046FFF766FF002020647DE75D
:103D5000206B012876D105F01000002872D006F003
:103D600010000028FAD000BF0020009020680068F2
:103D7000009020684068009000BF00BF2068406944
:103D800000F0400040285ED1A06B006840681FFA38
:103D900080F8B8F1000F54D0A08D404551DDA4F853
:103DA0002E80A06BC069B0F5807F43D000BF00BFFC
:103DB00021680C3151E8001F21F4807021680C311A
:103DC00041E80002002AF3D100BF00BF00BF216814
:103DD000143151E8001F21F001002168143141E83D
:103DE0000002002AF3D100BF00BF00BF21681431D8
:103DF00051E8001F21F040002168143141E8000221
:103E0000002AF3D100BF202084F83E000020206368
:103E100000BF00BF21680C3151E8001F21F01000E5
:103E200021680C3141E80002002AF3D100BFA06BE9
:103E3000FDF72CFAA08DE28D801A81B22046FFF7A3
:103E4000E9FE03E740E0A08DE18D401A1FFA80F8FB
:103E5000E08DC0B3B8F1000F35D000BF00BF2168BE
:103E60000C3151E8001F21F4907021680C3141E8B9
:103E70000002002AF3D100BF00BF00BF2168143147
:103E800051E8001F21F001002168143141E80002CF
:103E9000002AF3D100BF202084F83E0000202063D8
:103EA00000BF00BF21680C3151E8001F21F0100055
:103EB00021680C3141E80002002AF3D100BF4146DD
:103EC0002046FFF7A7FEC1E605F0800030B106F0FE
:103ED000800018B1204601F099FCB7E605F04000DB
:103EE00030B106F0400018B1204601F0EDFAADE621
:103EF00000BFABE64954000810B504460CB90120D8
:103F000010BDA06900B100E000BF94F83D0028B9E1
:103F1000002084F83C00204600F028F8242084F893
:103F20003D002068C06820F400502168C860204629
:103F300001F056FB2068006920F490402168086178
:103F40002068406920F02A00216848612068C06824
:103F500040F400502168C86000202064202084F8CC
:103F60003D0084F83E000020CAE7000010B586B08E
:103F70000446142101A8FCF7CFF95D492068884266
:103F800039D100BF002000905A48006840F400205A
:103F9000584908600846006800F40020009000BFFF
:103FA00000BF00BF0020009052481038006840F069
:103FB00004005049103908600846006800F0040009
:103FC000009000BF00BF4FF44060019002200290BB
:103FD00000200390032004900820059001A9464882
:103FE000FDF79EFB002205213420FDF76FFD3420F4
:103FF000FDF75CFD79E041492068884238D100BF77
:10400000002000903B48006840F4003039490860C7
:104010000846006800F40030009000BF00BF00BFF9
:104020000020009033481038006840F00800314903
:10403000103908600846006800F00800009000BFD2
:1040400000BF602001900220029000200390032016
:1040500004900720059001A92948FDF761FB002283
:1040600005212620FDF732FD2620FDF71FFD3CE04F
:1040700024492068884238D100BF002000901D48A4
:10408000006840F480201B4908600846006800F47E
:104090008020009000BF00BF00BF002000901548A6
:1040A0001038006840F002001249103908600846D4
:1040B000006800F00200009000BF00BF4FF44060B5
:1040C000019002200290002003900320049007201A
:1040D000059001A90C48FDF723FB002205212720AC
:1040E000FDF7F4FC2720FDF7E1FC06B010BD000051
:1040F000004C0040403802400008024000440040AC
:10410000000C0240004800400004024070472DE9C6
:10411000F84F04460E46174699464FF0000A94F8A9
:104120003D0020285AD106B117B90120BDE8F88F0B
:1041300000BF94F83C00012801D10220F6E70120DD
:1041400084F83C0000BF00202064212084F83D005A
:10415000FDF7F8FB8246A784E784A068B0F5805F8E
:1041600004D1206910B90025B04602E035464FF071
:10417000000800BF002084F83C0000BF1BE053464D
:10418000002280212046CDF8009001F06FFB08B19D
:104190000320CBE745B9B8F80000C0F30800216858
:1041A000486008F1020803E02878216848606D1C27
:1041B000E08C401EE084E08C0028E0D153460022D1
:1041C00040212046CDF8009001F050FB08B10320BB
:1041D000ACE7202084F83D000020A7E70220A5E7F7
:1041E000704700BFFEE700001FB50020009001905F
:1041F000029003905248534908604FF48030486061
:10420000002150488160012101610176002180F880
:104210002010C1624C4981620021C1600C21C16142
:10422000012180F830104161FCF7D0FC08B1FCF7A7
:10423000FFFB0020009001200190072002906946BA
:104240004048FCF7F9FB08B1FCF7F2FB01200090B5
:104250000220019069463B48FCF7EEFB08B1FCF7F1
:10426000E7FB022000900320019069463548FCF7E7
:10427000E3FB08B1FCF7DCFB032000900420019075
:1042800069463048FCF7D8FB08B1FCF7D1FB0620A3
:1042900000900520019069462A48FCF7CDFB08B143
:1042A000FCF7C6FB072000900620019069462548D0
:1042B000FCF7C2FB08B1FCF7BBFB0A20009007200B
:1042C000019069461F48FCF7B7FB08B1FCF7B0FB4B
:1042D0000B2000900820019069461A48FCF7ACFBBF
:1042E00008B1FCF7A5FB0C2000900920019069465D
:1042F0001448FCF7A1FB08B1FCF79AFB0D200090D5
:104300000A20019069460F48FCF796FB08B1FCF7BC
:104310008FFB0E2000900B20019069460948FCF7A6
:104320008BFB08B1FCF784FB0F2000900C20019060
:1043300069460448FCF780FB08B1FCF779FB1FBD18
:1043400000200140200300200100000F1FB50020C5
:1043500000900190029003901B481C4908604FF4A4
:104360008030486000211948816001210161017697
:10437000002180F82010C162154981620021C160CE
:104380000221C161012180F830104161FCF71EFC5F
:1043900008B1FCF74DFB082000900120019000209F
:1043A000029069460948FCF747FB08B1FCF740FB5F
:1043B000092000900220019069460448FCF73CFB6C
:1043C00008B1FCF735FB1FBD002101406803002048
:1043D0000100000F1FB50020009001900290039093
:1043E0003C483D4908604FF48030486000213A481D
:1043F0008160012101610176002180F82010C162F5
:10440000364981620021C1600821C161012180F823
:1044100030104161FCF7DAFB08B1FCF709FB04201E
:104420000090012001900720029069462A48FCF77D
:1044300003FB08B1FCF7FCFA052000900220019074
:1044400069462548FCF7F8FA08B1FCF7F1FA0620AE
:1044500000900320019069461F48FCF7EDFA08B16F
:10446000FCF7E6FA072000900420019069461A48FC
:10447000FCF7E2FA08B1FCF7DBFA0820009005200F
:10448000019069461448FCF7D7FA08B1FCF7D0FA56
:10449000092000900620019069460F48FCF7CCFAED
:1044A00008B1FCF7C5FA0E2000900720019069467C
:1044B0000948FCF7C1FA08B1FCF7BAFA0F200090DE
:1044C0000820019069460448FCF7B6FA08B1FCF7E9
:1044D000AFFA1FBD00220140B00300200100000F11
:1044E0001CB50020009001900E480F490860084656
:1044F000FCF71EFE08B1FCF79BFA0020009001902B
:10450000002269460848FCF79CFD08B1FCF790FAC8
:10451000102269460448FCF794FD08B1FCF788FABC
:104520001CBD0000007400403005002008B500BF2D
:10453000002000902248006840F480002049086074
:104540000846006800F48000009000BF00BF00BF74
:10455000002000900846006840F4001008600846FB
:10456000006800F40010009000BF00BF0022052189
:104570000E20FDF7ABFA0E20FDF798FA0022052178
:104580000F20FDF7A3FA0F20FDF790FA0022052176
:104590003820FDF79BFA3820FDF788FA0022052124
:1045A0003920FDF793FA3920FDF780FA0022052122
:1045B0003A20FDF78BFA3A20FDF778FA08BD0000A3
:1045C0003038024000B5A7B000202590269025A8DD
:1045D00004F0DAF823490860002023902490012198
:1045E00023A804F0DEF8204908601C221F491CA8FB
:1045F000FBF779FE00211CA804F0F8F81C490860BC
:104600001C221A491C3115A8FBF76DFE002115A8C4
:1046100004F0ECF8174908601C22144938310EA840
:10462000FBF761FE00210EA804F0E0F812490860D3
:104630001C220E49543107A8FBF755FE002107A89C
:1046400004F0D4F80D4908601C220849703168460E
:10465000FBF749FE0021684604F0C8F808490860E5
:1046600027B000BD140000201800002030A0000872
:104670000000002004000020080000200C000020A2
:104680001000002000B587B0142102A8FBF744FEFB
:1046900000BF00200190AB48006840F01000A9491D
:1046A00008600846006800F01000019000BF00BFDD
:1046B00000BF002001900846006840F0200008601C
:1046C0000846006800F02000019000BF00BF00BF56
:1046D000002001900846006840F08000086008460D
:1046E000006800F08000019000BF00BF00BF002004
:1046F00001900846006840F0040008600846006821
:1047000000F00400019000BF00BF00BF0020019036
:104710000846006840F0010008600846006800F0A4
:104720000100019000BF00BF00BF002001900846BB
:10473000006840F0020008600846006800F00200CF
:10474000019000BF00BF00BF002001900846006834
:1047500040F0080008600846006800F0080001907A
:1047600000BF00BF00BF002001900846006840F075
:10477000400008600846006800F04000019000BF5B
:1047800000BF002230217048FDF7D6F8002246F223
:1047900004016E48FDF7D0F8012211036C48FDF7C3
:1047A000CBF8012242F601216A48FDF7C5F8002244
:1047B0004FF480516748FDF7BFF8012244F20441ED
:1047C0006548FDF7B9F8002248F208016248FDF794
:1047D000B3F8012211036148FDF7AEF80022102161
:1047E0005B48FDF7A9F830200290012003900020DB
:1047F0000490059002A95448FCF792FF46F2040089
:1048000002900120039000200490059002A94F48D7
:10481000FCF786FF4FF4C050029000200390012067
:10482000049002A94948FCF77BFF4FF480500290A6
:1048300011200390012004900020059002A9444813
:10484000FCF76EFF40F204500290002003900490A9
:1048500002A94048FCF764FF40F2012002900120C9
:10486000039000200490059002A93A48FCF758FFF5
:104870004FF460500290112003900120049000201A
:10488000059002A93348FCF74BFF44F20C0002905C
:1048900011200390012004900020059002A92E48C9
:1048A000FCF73EFF4FF4807002900020039001203F
:1048B000049002A92948FCF733FF4FF4806002906E
:1048C000002003900120049002A92548FCF728FF4E
:1048D0004FF480500290112003900120049000209A
:1048E000059002A91D48FCF71BFF4FF400700290D1
:1048F00000200390049002A91748FCF711FF4FF421
:10490000044002900120039000200490059002A929
:104910001148FCF705FF10200290012003900020B1
:104920000490059002A90A48FCF7FAFE01200290C3
:1049300000200390049002A90348FCF7F1FE07B0A1
:1049400000BD000030380240001002400014024058
:1049500000040240000C024000180240000802401F
:104960000000024010B50F480F4908604FF48270F4
:10497000486000210C488160C160016141614FF4D1
:10498000007181613821C161802101620021416291
:1049900081620A21C162FDF79BFC08B1FCF748F86F
:1049A00010BD0000003001404405002010B50E4845
:1049B0000E4908604FF48270486000210B48816006
:1049C000C160016141614FF4007181613821C161B1
:1049D00000210162416281620A21C162FDF778FC17
:1049E00008B1FCF725F810BD003800409C050020F8
:1049F0001FB50020009001900290039014481549C3
:104A00000860532048600021124881604FF6FF7112
:104A1000C160002101618161FDF7C4FF08B1FCF7AD
:104A200007F80C48FEF763FB08B1FCF701F8022019
:104A3000009001200190002002900390002269461E
:104A40000448FEF7E5FA08B1FBF7F2FF1FBD0000CE
:104A500000440140D407002000B587B01C216846FF
:104A6000FBF75AFC1648174908605320486000219C
:104A70001448816044F61F61C160002101618021FA
:104A80008161FDF78FFF08B1FBF7D2FF0D48FEF7FC
:104A90001AFE08B1FBF7CCFF6020009000200190C7
:104AA00002900490002269460648FEF78AFD08B18C
:104AB000FBF7BEFF0348FEF72BFD07B000BD00006B
:104AC000004801401C08002000B58BB0242102A83A
:104AD000FBF722FC0020009001901848184908605C
:104AE000002048600021164881604FF6FF71C160C8
:104AF0000021016141618161012002900020039049
:104B00000120049000200590069007900120089055
:104B1000002009900A9002A90948FEF74CF808B154
:104B2000FBF786FF00200090019069460448FDF7DE
:104B3000DFFE08B1FBF77CFF0BB000BD00000140B9
:104B4000B406002000B58BB0242102A8FBF7E4FBDB
:104B50000020009001901848184908600020486023
:104B60000021164881604FF6FF71C160002101618C
:104B70008161012002900020039001200490002018
:104B800005900690079001200890002009900A9057
:104B900002A90A48FEF70FF808B1FBF749FF002009
:104BA0000090019069460548FDF7A2FE08B1FBF7A9
:104BB0003FFF0BB000BD000000040040FC060020D9
:104BC00000B589B00020079008901C216846FBF7CB
:104BD000A3FB1E481E4908605320486000211C4862
:104BE000816040F2E731C160002101618021816173
:104BF000FEF769FD08B1FBF71BFF00200790089046
:104C000007A91348FDF774FE08B1FBF711FF6020F8
:104C1000009040F2F31001900020029004200490D4
:104C2000082269460A48FEF7CCFC08B1FBF700FFF2
:104C30000C2269460648FEF7C4FC08B1FBF7F8FEF3
:104C40000348FEF765FC09B000BD00000008004005
:104C5000440700201FB500200090019002900390AF
:104C60001148124908605320486000210F488160B4
:104C70004FF6FF71C160002101618161FEF737FAD3
:104C800008B1FBF7D5FE0220009001200190002022
:104C900002900390042269460448FEF7B9F908B16E
:104CA000FBF7C6FE1FBD0000004001408C0700203E
:104CB00010B50B480B4908604FF4165048600021AE
:104CC00008488160C16001610C214161002181615E
:104CD000C161FFF711F908B1FBF7AAFE10BD000092
:104CE000004C00406408002010B50B480B490860D8
:104CF0004FF416504860002108488160C16001618E
:104D00000C21416100218161C161FFF7F5F808B113
:104D1000FBF78EFE10BD000000440040A8080020F4
:104D200010B50B480B4908604FF41650486000213D
:104D300008488160C16001610C21416100218161ED
:104D4000C161FFF7D9F808B1FBF772FE10BD000092
:104D500000480040EC08002000BFFEE700BFFEE76F
:104D60007CB504460D461646164800681821B0FB6F
:104D7000F1F01549B0FBF1F04FF47A71484301901E
:104D80006068B0F5827F0DD12B460022802120463D
:104D9000009600F01BF898B1606D40F0200060654F
:104DA00003207CBD00BF019800B908E00198401EB7
:104DB000019020688068C0F3C0100028F3D100BFC4
:104DC0000020EEE72C00002040420F002DE9F84FB4
:104DD00004460D4690461E46DDF82890FCF7B2FDCD
:104DE000A0EB0900371AFCF7ADFD82462C4800689D
:104DF000C0F3CB307843009045E0701C002842D0CF
:104E0000FCF7A0FDA0EB0A00B84200D2A7BB2068C7
:104E1000406820F0E000216848606068B0F5827F5B
:104E20000DD1A068B0F5004F03D0A068B0F5806F39
:104E300005D12068006820F0400021680860A06A61
:104E4000B0F5005F0DD100BF2068006820F400506D
:104E5000216808602068006840F4005021680860FC
:104E600000BF012084F8510000BF002084F85000EA
:104E700000BF0320BDE8F88FFFE7009800B90027C6
:104E80000098401E0090206880682840A84201D108
:104E9000012000E000204045AFD10020EAE70000FB
:104EA0002C00002000BF04210348FCF73BFD4FF419
:104EB000FA7003F058FCF6E70014024010B500BF8A
:104EC000502080F31188BFF34F8FBFF36F8F00BF67
:104ED00004F0D8FE18B14FF080500449086000BFBC
:104EE000002080F3118800BF10BD000004ED00E039
:104EF00000B593B0302107A8FBF70EFA142102A8E1
:104F0000FBF70AFA00BF002001902448006840F037
:104F10008050224908600846006800F080500190E7
:104F200000BF00BF00BF002001901D48006840F492
:104F300080401B4908600846006800F480400190EA
:104F400000BF00BF0220079001200A9010200B90A4
:104F500002200D9000210E9110210F914FF4A871A5
:104F6000109104211191129107A8FCF763FF08B179
:104F7000FBF75EFD0F2002900220039000200490BA
:104F80004FF4805005900690022102A8FCF7F0FD36
:104F900008B1FBF74DFD13B000BD000040380240E2
:104FA000007000400348006840F470000149086048
:104FB0007047000088ED00E010B50348FEF7DCF90B
:104FC0000248FEF7D9F910BDB40600208C07002076
:104FD00010B50348FEF7D0F90248FEF7CDF910BD31
:104FE000B4060020D407002010B50948FEF7C4F924
:104FF00008480078F02803D1074803F0FAF806E0E3
:10500000044800780F2802D1044803F0F2F810BDDC
:10501000440700209800002098460020D846002031
:1050200010B50548007910B10348FCF73CF8034877
:10503000FEF7A2F910BD0000300500203009002065
:1050400010B50268294B98420ED0B0F1804F0BD0BA
:10505000274B984208D0274B984205D0264B9842C0
:1050600002D0264B984203D122F070024B681A43BB
:105070001E4B984220D0B0F1804F1DD01C4B98425F
:105080001AD01C4B984217D01B4B984214D01B4B84
:10509000984211D01A4B98420ED01A4B98420BD01E
:1050A000194B984208D0194B984205D0184B98429A
:1050B00002D0184B984203D122F44072CB681A43B5
:1050C00022F080034C6943EA040202608B68C362E9
:1050D0000B688362054B984202D0084B984201D17D
:1050E0000B6903630123436110BD00000000014010
:1050F0000004004000080040000C00400004014093
:1051000000400140004401400048014000180040B8
:10511000001C00400020004030B501F01F050124B4
:1051200004FA05F3046A9C430462046A01F01F0553
:1051300002FA05F52C43046230BD000030B5056A63
:1051400025F001050562026A4368846924F0700451
:1051500024F003040D682C4322F002028D682A43D8
:10516000104DA84200D103E00F4DA84206D100BF68
:1051700022F00802CD682A4322F00402094DA84219
:1051800002D0094DA84207D123F4807323F40073A1
:105190004D692B438D692B43436084614D684563A2
:1051A000026230BD000001400004014030B5056AD4
:1051B00025F010050562026A4368846924F4E0441E
:1051C00024F440740D6844EA052422F020028D681E
:1051D00042EA0512124DA84200D103E0114DA84247
:1051E00007D100BF22F08002CD6842EA051222F00A
:1051F00040020B4DA84202D00A4DA84209D123F427
:10520000806323F400634D6943EA85038D6943EAB3
:105210008503436084614D688563026230BD000090
:10522000000001400004014030B5056A25F4807596
:105230000562026A4368C46924F0700424F0030420
:105240000D682C4322F400728D6842EA0522124D4B
:10525000A84200D103E0114DA84207D100BF22F4BB
:105260000062CD6842EA052222F480620A4DA8421B
:1052700002D00A4DA84209D123F4805323F40053ED
:105280004D6943EA05138D6943EA05134360C46120
:105290004D68C563026230BD00000140000401405A
:1052A00030B5056A25F480550562036A4468C26911
:1052B00022F4E04222F440720D6842EA052223F40F
:1052C00000538D6843EA0533084DA84202D0084DCB
:1052D000A84204D124F480444D6944EA8514446012
:1052E000C2614D680564036230BD000000000140EA
:1052F0000004014070B50C461546066A26F001060A
:1053000006628169026A184EB04214D0B0F1804F33
:1053100011D0164EB0420ED0154EB0420BD0154EE5
:10532000B04208D0144EB04205D0144EB04202D064
:10533000134EB04201D1012600E000261EB121F03B
:105340000301294301E041F0010121F0F001F026C1
:1053500006EA0316314322F00A0204F00A06324339
:105360008161026270BD0000000001400004004045
:1053700000080040000C00400004014000400140D3
:105380000018004070B50C461546066A26F0100657
:1053900006628169026A21F4407141EA052121F423
:1053A00070414FF4704606EA0336314322F0A00202
:1053B000A02606EA041632438161026270BD70B510
:1053C0000C461546066A26F480760662C169026AB2
:1053D00021F00301294321F0F001F02606EA03162B
:1053E000314322F420624FF4206606EA0426324359
:1053F000C161026270BD70B50C461546066A26F49E
:1054000080560662C169026A21F4407141EA0521B1
:1054100021F470414FF4704606EA0336314322F41A
:1054200020424FF4204606EA04363243C16102624C
:1054300070BD000010B50348FEF7EEFB014802F016
:10544000DDFD10BD6408002070B50546AC6B002082
:10545000E085E0842046FEF7DEFB70BD00BF00BFA4
:1054600002680C3252E8002F22F4907102680C326C
:1054700042E80013002BF3D100BF00BF00BF026859
:10548000143252E8002F22F001010268143242E87F
:105490000013002BF3D100BF016B01290ED100BF17
:1054A00000BF02680C3252E8002F22F0100102689F
:1054B0000C3242E80013002BF3D100BF202180F80A
:1054C0003E1000210163704710B504462068C06893
:1054D00020F040002168C860202084F83D0020466C
:1054E000FEF77EFE002010BDF8B5044694F83E009D
:1054F000222873D1A068B0F5805F0CD1206950B923
:105500000025A66A20684068C0F308003080A06AC1
:10551000801CA06215E0A56A0026A068B0F5805F37
:1055200003D0A06828B9206918B92068406828709D
:1055300004E02068406800F07F002870A06A401CEA
:10554000A062E08D401E80B2E085002844D1206832
:10555000C06820F020002168C8602068C06820F47E
:1055600080702168C8602068406920F001002168CF
:105570004861202084F83E00206B012826D10020BD
:10558000206300BF00BF21680C3151E8001F21F0EB
:10559000100021680C3141E80002002AF3D100BF5D
:1055A0002068006800F0100010280AD100BF002019
:1055B000009020680068009020684068009000BF5C
:1055C00000BFA18D2046FEF725FB02E02046FEF736
:1055D0009DFD0020F8BD01E00020FBE70220F9E777
:1055E0002DE9F84F04462068006920F44050E16836
:1055F0000843216808612169A0680843616908437C
:10560000E169084300902068C06849F20C61884352
:10561000009908432168C8602068406920F4407000
:10562000A16908432168486176492068884203D00F
:1056300075492068884203D1FCF794FB814602E05B
:10564000FCF780FB8146E069B0F5004F6CD1022089
:105650006168A0FB015003461920A9FB00700146B8
:105660002A463846FAF70EFE6421B0FBF1F04FEA05
:10567000001A02206168A0FB01510B461920A9FB0A
:1056800000712A463846FAF7FDFD8346022061681C
:10569000A0FB015003461920A9FB00712A46384699
:1056A000FAF7F0FD6421B0FBF1F000EBC00101EB73
:1056B0000010ABEB8000322101EBC0006421B0FB95
:1056C000F1F000F0F8000AEB400A02206168A0FB4C
:1056D000015003461920A9FB007001462A463846AE
:1056E000FAF7D0FD834602206168A0FB0150034613
:1056F0001920A9FB00712A463846FAF7C3FD642138
:10570000B0FBF1F000EBC00101EB0010ABEB80004F
:10571000322101EBC0006421B0FBF1F000F0070082
:105720005044216888606AE004206168A0FB015051
:1057300003461920A9FB007001462A463846FAF7AD
:10574000A1FD824604206168A0FB01500346192098
:10575000A9FB007001462A463846FAF793FD6421FA
:10576000B0FBF1F000EBC00101EB0010AAEB8000F0
:10577000322101EB00106421B0FBF1F000F0F00ADF
:1057800004206168A0FB017003461920A9FB0051A9
:105790003A462846FAF776FD6421B0FBF1F00AEBB1
:1057A000001A04206168A0FB01510B461920A9FBD7
:1057B00000712A463846FAF765FD83460420616881
:1057C000A0FB015003461920A9FB007001462A46A0
:1057D0003846FAF757FD6421B0FBF1F000EBC00149
:1057E00001EB0010ABEB8000322101EB00106421D3
:1057F000B0FBF1F000F00F00504421688860BDE874
:10580000F88F00000010014000140140014691F89B
:105810003D00212828D18868B0F5805F0BD1086948
:1058200048B90A6A1088C0F308000B685860086A13
:10583000801C086205E00B6A581C086218780B6827
:105840005860C88C401E80B2C88458B90868C068C7
:1058500020F080000B68D8600868C06840F0400005
:105860000B68D860002070470220FCE72DE9F0416A
:1058700004460D4617469846069E34E0701C88B3D1
:105880002EB1FCF75FF8A0EB0800B0422BD900BFA7
:1058900000BF21680C3151E8001F21F4D07021684D
:1058A0000C3141E80002002AF3D100BF00BF00BF65
:1058B0002168143151E8001F21F0010021681431E2
:1058C00041E80002002AF3D100BF202084F83D0007
:1058D00084F83E0000BF002084F83C0000BF032095
:1058E000BDE8F081FFE7206800682840A84201D1A8
:1058F000012000E00020B842C0D00020F0E7000006
:1059000010B50348FEF788F9014802F077FB10BD97
:10591000A808002010B50348FEF77EF9014802F000
:105920006DFB10BDEC08002000BFFEE702480068D8
:10593000C0F30220704700000CED00E010B5002815
:1059400004DB0A07130E054A135406E00A07140E77
:10595000034A00F00F031B1FD45410BD00E400E005
:1059600018ED00E02DED020B019820F000400190B1
:105970009DED000B02B0704702E008C8121F08C17D
:10598000002AFAD170477047002001E001C1121FC0
:10599000002AFBD17047000011B526E0009CB4F549
:1059A000617F02D94FF4617400E0009C23464FF000
:1059B000E024A069542404FB1301002908DB00BF84
:1059C0004FF0E024A26982420CDA8A42F8DA09E058
:1059D000084C214400BF4FF0E024A2698242FADD66
:1059E0008A42F8DC009CE41A0094009C002CD5D17B
:1059F00018BD0000204801002DE9F05F044614B9ED
:105A00000020BDE8F09F2668A788D4F80880B4F885
:105A10000C902569D4F814A04FF0000B72B6012247
:105A200039463046A8470A20FFF7B6FF002239461C
:105A30003046A8474FF4FA70FFF7AEFF012239460F
:105A40003046A8473220FFF7A7FF012249464046CB
:105A5000D047012800D18346012239463046A84765
:105A6000F020FFF799FF62B65846CAE72DE9F84FD4
:105A7000044614B90020BDE8F88FD4F80080B4F8CB
:105A80000490D4F808A0A08900902569D4F814B037
:105A9000002672B6002722E0002249464046A84769
:105AA0000520FFF779FF012249464046A8470A2012
:105AB000FFF772FF7610012250460099D84701285F
:105AC00001D146F080063220FFF766FF01224946E9
:105AD0004046A8470520FFF75FFF781CC7B2082F94
:105AE000DADB62B63046C6E72DE9F0472DED068BCE
:105AF00081460C46B9F1000F03D1BDEC068BBDE821
:105B0000F08700254846216A8847012804D19FED87
:105B1000380A84ED070AF0E7CC214846626A9047CC
:105B200044214846626A90474846216A8847CC210A
:105B30004846626A9047BE214846626A9047484696
:105B4000A16A884707464846A16A88470646072E45
:105B500006DDF043C6B2F843C7B24FF0010801E0DA
:105B60004FF0000835462D023D444FF6FF70854248
:105B700003D015B1B5F5C86F00D3BEE72846FAF7D4
:105B800048FC41EC190B9FED1B0B53EC102BFAF763
:105B9000CEFB41EC180BFAF78DFCE061B8F1000F79
:105BA00014D02846FAF735FC41EC1A0B9FED110B87
:105BB00053EC102BFAF7BBFB41EC190B81F00041C1
:105BC00041EC180BFAF776FCE0610FE02846FAF793
:105BD00020FC41EC190B9FED070B53EC102BFAF74F
:105BE000A6FB41EC180BFAF765FCE06100BF84E707
:105BF00000000000000000000000B03F2DE9F04769
:105C000004460E460CB9BDE8F087D4F80080B4F81D
:105C10000490256972B600271FE0002249464046DD
:105C2000A8470520FFF7B8FE06F0010020B10122C9
:105C300049464046A84703E0002249464046A84757
:105C40004620FFF7A9FE012249464046A8477610A4
:105C50000520FFF7A1FE781CC7B2082FDDDB62B676
:105C600000BFD0E770B50246002318E0002011E025
:105C700052F82060451C52F82550AE4209D952F81E
:105C80002040451C52F8255042F82050451C42F84F
:105C90002540401CCD1A6D1E8542E9D85B1C4D1E67
:105CA0009D42E3D870BD000070B5054605B970BDD2
:105CB00000242878F02801D1244C03E028780F280C
:105CC00000D1234C2348007901283CD1E07A0228F6
:105CD0000BD12049886800F0E5FA00201E490870C1
:105CE0001E4908700420E07214E0E07A032804D111
:105CF0001849886800F058FA0CE0A07A012803D10E
:105D00000020A072042600E0E67A1248816830463E
:105D100000F028F800200F49087194ED090AD4ED2D
:105D2000040AB0EE001A60EE810AB4EE600AF1EEE9
:105D300010FA01D0042E06D101200949087003F0A1
:105D40009BFF0749886000BFB1E70000984600202C
:105D5000D8460020B04800205C7700206C770020F7
:105D6000507700202DE9F05F2DED088B83460C461F
:105D70001CB9BDEC088BBDE8F09F002500264FF054
:105D80003D08A946DFEDF48AAA46F4480078F028D9
:105D900008D1DFF8CC93F34FF34890ED079AD9ED93
:105DA000089A0BE0ED4800780F2807D1DFF8BC9384
:105DB000EF4FF04890ED079AD9ED089A0522284652
:105DC000691CCDB222544FEA28222846691CCDB264
:105DD00022542846691CCDB204F8008000222846CF
:105DE000691CCDB22254B1222846691CCDB222547E
:105DF00000222846691CCDB22254A1222846691CE3
:105E0000CDB22254D54802782846691CCDB222541E
:105E10002846691CCDB204F800B0012672E00B2EB2
:105E200035DAD04800EB860090ED000ADFEDD20AAB
:105E300020EE200ADFEDD00A20EE200ADFEDCF0AA7
:105E400080EE201ABCEEC10A10EE100AC0F3072241
:105E50002846691CCDB22254C24800EB860090ED62
:105E6000000ADFEDC50A20EE200ADFEDC30A20EEAE
:105E7000200ADFEDC20A80EE201ABCEEC10A10EE45
:105E8000100AC2B22846691CCDB2225438E0A6F1ED
:105E90000A00B74901EB800090ED000ADFEDB60A79
:105EA00020EE200ADFEDB40A20EE200ADFEDB30A6F
:105EB00080EE201ABCEEC10A10EE100AC0F30722D1
:105EC0002846691CCDB22254A6F10A00A84901EB6C
:105ED000800090ED000ADFEDA80A20EE200ADFED39
:105EE000A60A20EE200ADFEDA50A80EE201ABCEEFD
:105EF000C10A10EE100AC2B22846691CCDB2225463
:105F0000701CC6B2152E8ADB012609E007EB86005D
:105F100090ED000A30EE280AF0EE408A701CC6B2FE
:105F20000B2EF3DBB2EE040AC8EE800AF0EE608AB4
:105F30009FED920AC8EE800AF0EE608ABCEEE80A95
:105F400010EE100A4FF47A714843C0F30722284636
:105F5000691CCDB22254BCEEE80A10EE100AE8210A
:105F60004843C2B22846691CCDB2225497ED000ABC
:105F7000DFED830A30EE600A10EE101A0846FAF7D9
:105F800055FA41EC1B0BB0EE4B0AF0EE6B0AFFF733
:105F9000E9FCB0EE40AAF0EE60AA9FED7A0B53EC5C
:105FA000102B51EC1A0BFAF755FA02D29FED778AB3
:105FB00053E097ED000ADFED760A30EE600A10EE4E
:105FC000101A0846FAF732FA41EC1B0BB0EE4B0AF6
:105FD000F0EE6B0AFFF7C6FCB0EE40AAF0EE60AA46
:105FE0009FED6C0B53EC102B51EC1A0BFAF732FAB5
:105FF00002D29FED678A30E097ED000ADFED670A75
:1060000030EE600A10EE101A0846FAF70FFA41EC6B
:106010001B0BB0EE4B0AF0EE6B0AFFF7A3FCB0EEE1
:1060200040AAF0EE60AA9FED5B0B53EC102B51ECF5
:106030001A0BFAF70FFA02D29FED588A0DE097ED8E
:10604000000AF1EE080AB4EEE00AF1EE10FA02D20C
:106050009FED418A01E097ED008A9FED470A28EE07
:10606000000ABCEEC00A10EE100AC0F30722284650
:10607000691CCDB222549FED400A28EE000ABCEE06
:10608000C00A10EE100AC2B22846691CCDB22254D2
:10609000B5EEC09AF1EE10FA05D24FF0010AB1EE5A
:1060A000490AB0EE409A2846691CCDB204F800A017
:1060B0009FED3B0A29EE000ABCEEC00A10EE100A62
:1060C000C0F307222846691CCDB222549FED340A42
:1060D00029EE000ABCEEC00A10EE100AC2B2284631
:1060E000691CCDB222549FED240A29EE800ABCEE31
:1060F000C00A10EE100AC0F307222846691CCDB270
:1061000022549FED1D0A29EE800ABCEEC00A10EE53
:10611000100AC2B22846691CCDB222540122284678
:10612000691CCDB22254CD222846691CCDB222541E
:1061300040222846691CCDB222541B222846691CE5
:10614000CDB222544FF6FF732A4621461548FDF77B
:10615000DEFF00BF0DE600000000000098000020F8
:106160009846002094740020FC4F0020D846002060
:10617000C07400202850002000007A4400007A43B8
:10618000A470DD40000000403333C33F3D0ADF40D0
:1061900033330341000000A09999B93FEC511041FD
:1061A0000000C842D848002070B5044604B970BD4C
:1061B00000250F26052229466D1C625432122946FD
:1061C0006D1C625429466D1C6654002229466D1CC4
:1061D0006254B12229466D1C6254002229466D1C6E
:1061E0006254A12229466D1C62542A48027828462E
:1061F000691CCDB2225403222846691CCDB2225418
:10620000254890ED030ABCEEC00A10EE100AC0F358
:1062100007222846691CCDB222541F4890ED030A7C
:10622000BCEEC00A10EE100AC2B22846691CCDB2FC
:1062300022541A4890ED030ABCEEC00A10EE100A70
:10624000C0F307222846691CCDB22254134890EDB2
:10625000030ABCEEC00A10EE100AC2B22846691C3E
:10626000CDB2225400222846691CCDB222544022CD
:106270002846691CCDB222541B222846691CCDB287
:1062800022544FF6FF732A4621460548FDF73FFF8B
:1062900000BF8CE798000020F476002018770020DB
:1062A000D848002070B5044604B970BD00254726C3
:1062B000052229466D1C6254321229466D1C625417
:1062C00029466D1C6654002229466D1C6254B12279
:1062D00029466D1C6254002229466D1C6254A1227D
:1062E00029466D1C6254454802782846691CCDB287
:1062F000225402222846691CCDB2225400201CE000
:106300003F4931F820103E4A783A32F82020891A65
:10631000C1F3072329466A1CD5B26354384911F8E2
:106320002010374A783A12F82020891ACBB2294631
:106330006A1CD5B26354411CC8B20A28E0DB0020B5
:106340001CE0304931F820102E4A783A32F82020EB
:10635000891AC1F3072329466A1CD5B26354294917
:1063600011F82010274A783A12F82020891ACBB267
:1063700029466A1CD5B26354411CC8B20A28E0DB26
:1063800000200EE01E49283911F82020283911F884
:106390002010511ACBB229466A1CD5B26354411C55
:1063A000C8B20A28EEDB00200EE01649283911F8A1
:1063B0002020283911F82010511ACBB229466A1C26
:1063C000D5B26354411CC8B20A28EEDBCD22284660
:1063D000691CCDB2225440222846691CCDB22254F9
:1063E0001B222946681CC5B262544FF6FF732A4629
:1063F00021460548FDF78BFE00BF56E798000020B8
:106400006475002004760020D848002070B5054649
:1064100005B970BD05F10C0420780022114602F088
:10642000F7F820780F4A6C2102F0F2F82078212248
:106430000A2102F0EDF8207800220B2102F0E8F8A2
:106440002078094A102102F0E3F82078074A7021E9
:1064500002F0DEF820780722012102F0D9F800BF0F
:10646000D7E70000530141001F1F07001E264CC440
:10647000F0B5014601B9F0BD0A464B1C8C1C01F178
:106480001E00058865B105886D1E05800588642697
:1064900095FBF6F706FB17553DB901251D7004E085
:1064A00041F28835058001251D701578012D04D134
:1064B00041F2883505800125257000BFDBE700002B
:1064C0002DE9F04105460DB9BDE8F0812E466F1C5F
:1064D00005F102082C1D284600F004FAB8F8000067
:1064E00000F08EFA206039780C4A515C206808432D
:1064F0002060206820F4706020600021304600F0A9
:1065000011F86423042221460548FCF703F8012111
:10651000304600F007F800BFD6E70000DCA0000816
:106520004405002070B505460C4605B970BD2878B5
:1065300001280ED1012C05D1012210210F48FBF7B3
:10654000FBF918E0BCB9002210210C48FBF7F4F964
:1065500011E0287802280ED1012C05D101228103F7
:106560000748FBF7E9F906E02CB900224FF4004197
:106570000348FBF7E1F900BFD8E700000004024040
:106580000018024010B504461148007800B910BD4B
:106590000F4844600F48C08A002803DD03F06CFBFD
:1065A0000B49886003F068FB09498968084A52680A
:1065B0001144884205D2012220210748FBF7BCF98B
:1065C00004E0002220210448FBF7B6F900BFDEE713
:1065D00050770020B04800200010024010B504465B
:1065E00004B910BD0A4802F079F80A4802F076F8BA
:1065F0002146074801F07AFD2146064801F076FD64
:10660000204600F055FB204601F0C4FF00BFE8E73C
:1066100018770020F476002010B5044604B910BDA8
:10662000204600F0DEF9204601F0C0FC204600F0D4
:10663000A5FA204601F0BCFD204601F0CDFE00BFCA
:10664000EDE700002DE9F04104460025A8460027AB
:106650000026608842F21071884202DD08466080A0
:1066600006E0608841F28831884201DA084660809D
:106670006088A0F59850883885B204F10408A8F81D
:1066800000500DB9002700E00127C5EB053041F2AD
:10669000883190FBF1F086B21E480088864203DB09
:1066A0001C480088301A86B21B48844216D12FB18C
:1066B000012291031948FBF73FF905E000224FF44E
:1066C00080411648FBF738F900211548FAF7A2FD7A
:1066D0003346002211461248FAF786FD11488442DB
:1066E00016D12FB1012251030C48FBF725F905E023
:1066F00000224FF400510948FBF71EF91021084809
:10670000FAF788FD3346002210210548FAF76CFDA0
:10671000BDE8F0811C000020180500200014024094
:10672000300500202405002070B505460C46F02DEC
:106730000ED1012C05D1002209030E48FBF7FCF80D
:1067400016E0ACB9012211030A48FBF7F5F80FE097
:106750000F2D0DD1012C05D10022E1020648FBF7D7
:10676000EBF805E024B90122D1020348FBF7E4F875
:1067700070BD000000040240000C02402DE9F04111
:1067800007460C46154607B114B90020BDE8F08154
:106790004FF0000821463846FFF764FAEEB204E0F5
:1067A00057F826008044701CC6B2601BB042F7D870
:1067B000022000FB1540B8FBF0F0E7E710B500241D
:1067C00023E000200AE00C2101FB0041104A52F8AE
:1067D0002110104A42F82010411CC8B26428F2DB94
:1067E000052264210B48FFF7C9FF0B4941F824003B
:1067F000084650F8240040F69911884203D908460B
:10680000054941F82400601CC4B20C2CD9DB10BD32
:106810005450002004730020B472002010B50024EE
:1068200018E000200AE0022101FB00410B4A52F867
:1068300021100B4A42F82010411CC8B26428F2DB38
:10684000052264210648FFF799FF064941F8240014
:10685000601CC4B2022CE4DB10BD000014630020F5
:1068600004730020B400002010B5002423E00020B1
:106870000AE0082101FB0041104A52F82110104A99
:1068800042F82010411CC8B26428F2DB05226421C2
:106890000B48FFF773FF0B4941F82400084650F8F6
:1068A000240040F69911884203D90846054941F869
:1068B0002400601CC4B2082CD9DB10BD3466002053
:1068C00004730020E4720020F02802D1034AD17240
:1068D00003E00F2801D1024AD17270479846002088
:1068E000D846002000B97047134A904201D113499D
:1068F00003E0134A904200D112494A8842F2080349
:106900009A4202D10122427013E04A8841F63A339A
:106910009A4204D1002242800222427009E04A8851
:1069200042F23C339A4202D10322427001E000223B
:10693000427000BFD7E70000A40000201805002027
:10694000AC00002024050020F0B5054601B9F0BDDB
:106950004B1C881C0C1D8A1D861D2F683F68C7F3C1
:1069600000171F702F687F6A07800788B4F800C07F
:10697000674501DA012700E0002793F800C0BCF169
:10698000000F02D14FF0010C01E04FF0000C07EABC
:106990000C071FB117887F1C3FB217800788B4F817
:1069A00000C0674501DD012700E0002793F800C023
:1069B000BCF1010F02D14FF0010C01E04FF0000CCF
:1069C00007EA0C071FB117887F1E3FB217800788A0
:1069D00027800788B2F800C047EA0C47376000BF3D
:1069E000B5E710B50446204600F036F8204600F022
:1069F000C7F9204600F0A8F8204600F03BF910BD8A
:106A000030B50446012300220020002121E004EAE1
:106A1000030565B101221F25A5EB4105AA401043DE
:106A200001221E25A5EB4105AA4090430BE001225F
:106A30001F25A5EB4105AA40904301221E25A5EB89
:106A40004105AA4010434FF6FF7505EA43034D1C6C
:106A5000E9B20A29DBDB30BD2DE9F04704460CB969
:106A6000BDE8F087651DE61C271D04F106094FF0FF
:106A70000008244884420DD1DFF88C804FF48071E7
:106A80002248FAF747FF10B90120287012E00020D1
:106A900028700FE01E4884420CD1DFF878804FF454
:106AA00080611D48FAF736FF10B90120287001E017
:106AB000002028702878012803D099F800000128C8
:106AC0001BD198ED080AF2EE080AB4EEE00AF1EEE6
:106AD00010FA04DD002030700120387010E098EDCD
:106AE000080AF2EE080AB4EEE00AF1EE10FA07D254
:106AF000012030700020387002E0002030703870C3
:106B000000BFADE79846002018470020000802406B
:106B1000D8460020E447002000000240024692EDE3
:106B2000001AB4EEC01AF1EE10FA06D992ED001A6E
:106B3000B4EEE01AF1EE10FA02DB0120087001E079
:106B4000002008700878704700B97047C11D074AD7
:106B5000904203D1064AD2780A7005E0054A904275
:106B600002D1054AD2780A7000BFEEE798460020AD
:106B700018470020D8460020E44700202DE9F05FA8
:106B80002DED048B04461CB9BDEC048BBDE8F09FD1
:106B900004F10D0704F1140A04F1180B04F12405A3
:106BA0002E1F04F1280804F11C0994ED0B0AB5EE20
:106BB000C00AF1EE10FA00D1E6E799ED000AD5ED32
:106BC000000AB4EE600AF1EE10FA00D1DCE795EDB0
:106BD000000AD6ED000A30EE600A10EE101A0846E0
:106BE000F9F724FC41EC190BB0EE490AF0EE690A02
:106BF000FEF7B8FEB0EE408AF0EE608A51EC180B5A
:106C0000F9F758FCC8F8000098ED000AF7EE000A02
:106C100020EE200ADFED150A20EE200ADFED140A2F
:106C200020EE200ABCEEC00A8AED000A0020CBF854
:106C3000000095ED000AD6ED000AB4EEE00AF1EE90
:106C400010FA01DD38700AE095ED000AD6ED000A71
:106C5000B4EEE00AF1EE10FA01D20120387095EDA1
:106C6000000A89ED000A00BF8EE7000000004843DB
:106C70000000044400B970470021094A904201D144
:106C8000084903E0084A904200D1084991ED080AFA
:106C9000D0ED0B0A30EE600A80ED080A00BFEAE78B
:106CA0009846002018470020D8460020E4470020DE
:106CB00070B5014601B970BD01F10C00031D4C888F
:106CC0000A1D2A4D95ED050ABCEEC00A10EE105AB9
:106CD000274E758035466D8800EE105AB8EE400A92
:106CE000DFED240A80EE201A354685ED021A15885C
:106CF000A54208DD90ED000ADFED1F0A30EE200A04
:106D000080ED000A09E00025158090ED000ADFED16
:106D10001A0A30EE600A80ED000A90ED000AF1EEEA
:106D2000060AB4EEE00AF1EE10FA02D2B1EE060A5B
:106D30000DE090ED000AF2EE040AB4EEE00AF1EE86
:106D400010FA02DDB1EE060A01E090ED000A80EDD6
:106D5000000A90ED000ADFED090A20EE200ABCEEE1
:106D6000C00A10EE105A1D8000BFA4E7F476002080
:106D70003C770020000070426F12033A0000484345
:106D80002DE9FF5F04460CB9BDE8FF9F2078039012
:106D900004F10608D4F8309000253248844200D12E
:106DA000314D3248844200D1314D05F1140AD5F8F5
:106DB00008B0A81D0290861D371D039828B9002031
:106DC0003060002102980180DEE794ED080ADFEDD3
:106DD000290AB4EEE00AF1EE10FA07DB94ED0B0A93
:106DE000B5EEC00AF1EE10FA00D0CDE702F044FF94
:106DF000DAF800101E31884231D902F03DFFCAF89E
:106E000000003168ABEB0100002801DB014600E027
:106E100041423960306800B344F62060814505D1B5
:106E2000322001904FF4AF70009007E01248814586
:106E300004D1C82001904FF4167000903968019871
:106E4000814207D939680098814203D2002088F82E
:106E5000000002E0012088F80000C6F800B000BF82
:106E600092E700009846002068460020D84600209F
:106E700080460020CDCCCC3D80380100064890ED06
:106E8000000A064880ED020A054890ED000A054810
:106E900080ED020A7047000094740020180500205D
:106EA000C07400202405002010B5FFF787FCB2480D
:106EB00090ED0B0AB8EE400AF0EE040A20EE200A2C
:106EC000DFEDAE0A80EE201AAD4880ED011AAA4827
:106ED00090ED0A0AB8EE400AF0EE040A20EE200A0D
:106EE000DFEDA60A80EE201AA54880ED021AA2481E
:106EF00090ED050AB8EE400AF0EE040A20EE200AF2
:106F0000DFED9E0A80EE201A9D4880ED031A9A4814
:106F100090ED040AB8EE400AF0EE040A20EE200AD2
:106F2000DFED960A80EE201A954880ED041A92480B
:106F300090ED030AB8EE400AF0EE040A20EE200AB3
:106F4000DFED8E0A80EE201A8D4880ED051A8A4802
:106F500090ED020AB8EE400AF0EE040A20EE200A94
:106F6000DFED860A80EE201A854880ED061A8248F9
:106F700090ED010AB8EE400AF0EE040A20EE200A75
:106F8000DFED7E0A80EE201A7D4880ED071A7A48F0
:106F900090ED000AB8EE400AF0EE040A20EE200A56
:106FA000DFED760A80EE201A754880ED081A7248E7
:106FB00090ED090AB8EE400AF0EE040A20EE200A2D
:106FC000DFED6E0A80EE201A6D4880ED091A6A48DE
:106FD00090ED080AB8EE400AF0EE040A20EE200A0E
:106FE000DFED660A80EE201A654880ED0A1A6248D5
:106FF00090ED070AB8EE400AF0EE040A20EE200AEF
:10700000DFED5E0A80EE201A5E4880ED011A5A48D4
:1070100090ED060AB8EE400AF0EE040A20EE200ACF
:10702000DFED560A80EE201A564880ED021AFFF76F
:10703000F5FB554890ED010AB8EE400AF2EE040A5D
:1070400020EE200ADFED4D0A80EE201A4C4880ED3C
:10705000001A4D4890ED000AB8EE400AF2EE040A1C
:1070600020EE200ADFED450A80EE201A454880ED2B
:10707000001AFFF7F9FB454890ED040AB8EE400A04
:10708000F0EE040A20EE200ADFED3C0A80EE201A22
:107090003C4880ED031A3D4890ED030AB8EE400AE3
:1070A000F0EE040A20EE200ADFED340A80EE201A0A
:1070B000344880ED041A354890ED020AB8EE400AD3
:1070C000F0EE040A20EE200ADFED2C0A80EE201AF2
:1070D0002C4880ED051A2D4890ED010AB8EE400AC3
:1070E000F0EE040A20EE200ADFED240A80EE201ADA
:1070F000244880ED061A254890ED000AB8EE400AB3
:10710000F0EE040A20EE200ADFED1C0A80EE201AC1
:107110001C4880ED071A1D4890ED070AB8EE400A9A
:10712000F0EE040A20EE200ADFED140A80EE201AA9
:10713000144880ED081A154890ED060AB8EE400A8A
:10714000F0EE040A20EE200ADFED0C0A80EE201A91
:107150000C4880ED091A0D4890ED050AB8EE400A7A
:10716000F0EE040A20EE200ADFED040A80EE201A79
:10717000044880ED0A1A10BDB4720020000080455A
:1071800094740020C0740020B4000020E472002039
:1071900030B5014601B930BD01F11402901C002345
:1071A000154CA14200D1154B154CA14200D1154BF5
:1071B0001C7A012C10D100241C721488962C02DA3F
:1071C0009624148006E01488B4F57A7F02DD4FF42B
:1071D0007A7414801488048004881CB10488641EA6
:1071E000048001E0002404800488012C01D1064DB4
:1071F0002C7100BFCFE70000184700209846002000
:10720000E4470020D8460020B048002000B970476D
:107210000146002202604260064A904202D10122E9
:107220000A7004E0044A904201D102220A7000BFB1
:10723000EDE70000A4000020AC00002010B54FF4E2
:10724000966208490848F9F721FEC822074908480C
:10725000F9F71CFE4FF4487206490748F9F716FE85
:1072600010BD0000545000202003002014630020B3
:107270006803002034660020B003002010B50446E7
:1072800004B910BD18212046F9F746F80F4884428A
:1072900009D14FF48050A0800D4820600420A081C7
:1072A0000C48A0600BE00C48844208D14FF48040A9
:1072B000A0800A4820604015A0810848A0600848C6
:1072C00060610848206100BFDBE70000CC4F002070
:1072D00000080240000C0240E44F00200018024069
:1072E000151900083919000810B5044604B910BD75
:1072F0002C212046F9F710F80948844202D10120D8
:10730000207004E00748844201D102202070064822
:107310002062064860620648A06200BFE7E70000FE
:10732000FC4F002028500020F9590008FD5B0008A0
:107330006D5A000870B505460C4605B104B970BD1C
:1073400018212046F8F7E8FF3C212846FBF726FDE8
:107350000648854202D10120207004E0044885429D
:1073600001D10220207000BFE9E70000FC060020E8
:10737000B406002010B5044604B910BD24212046EF
:10738000F8F7CAFF1948FBF7A3FB00BF17480068CE
:10739000006A20F0A00015490968086213480068D7
:1073A000006A40F0200011490968086200BF04210A
:1073B0000E48FBF719FF0E48FBF78AFB00BF0C488D
:1073C0000068006A20F00A00094909680862084854
:1073D0000068006A40F0020005490968086200BFC1
:1073E00000210348FBF700FF00BFC6E78C07002021
:1073F000D40700202DE9F04704460CB9BDE8F0871A
:1074000004F1010A04F11E0504F11106771C04F1D0
:10741000180804F11A09CC212046F8F77DFF012055
:107420008AF8000041F28830288002203070032062
:1074300038700020A8F800001220A9F80000534876
:1074400084422FD12622524904F12800F8F74BFF3D
:107450004F48C18C4E20015304F128004C498A6AE0
:107460002265898DA4F854104948C18D56200153D6
:107470004748016BA165092200F1340104F15C0069
:10748000F8F731FF424890F83D1084F8651090F805
:107490003E1084F86610016CA1663E48A0603E482C
:1074A000E06064E03D4884422FD126223C4904F14B
:1074B0002800F8F718FF3A48C18C4E20015304F118
:1074C000280037498A6A2265898DA4F85410344807
:1074D000C18D562001533248016BA165092200F18C
:1074E000340104F15C00F8F7FEFE2D4890F83D10E1
:1074F00084F8651090F83E1084F86610016CA1665F
:107500002848A0602848E06031E0284884422ED115
:107510002622274904F12800F8F7E5FE2448C18C0B
:107520004E20015304F1280021498A6A2265898D81
:10753000A4F854101E48C18D562001531C48016BFD
:10754000A165092200F1340104F15C00F8F7CBFEDB
:10755000174890F83D1084F8651090F83E1084F8B4
:107560006610016CA1661348A0601348E060A06A31
:10757000C06840F02000A16AC860A06AC06840F0FE
:107580001000A16AC86000BF38E70000184700205B
:10759000640800207C4900207C4A0020E447002049
:1075A000A80800207C4B00207C4C0020B048002024
:1075B000EC0800207C4D00207C4E00200021016062
:1075C0004160816042F208014180704710B5044675
:1075D00004B910BD40212046F8F79EFE0E488442B3
:1075E00002D1F020207304E00C48844201D10F2026
:1075F000207300202070B0EE000A84ED040AE072CF
:107600003220606344F6206020630820E063204657
:10761000FEF7FCFE00BFDCE798460020D8460020BD
:107620002DE9F0472DED048B05461DB9BDEC048B0B
:10763000BDE8F08700244A480078F02803D1494F7C
:10764000494C4A4E06E0464800780F2802D1484F80
:10765000484C494E95F80980B8F1000F09D0B8F1AF
:10766000010F09D0B8F1020F09D0B8F1030F10D102
:107670000AE0002020700DE0012020700AE00120C7
:1076800060700020A07005E00120A07000206070F4
:1076900000E000BF00BF95F80A90B9F1000F00D0DC
:1076A00000BFB8F1020F0DDA687B297B40EA0120A8
:1076B00000EE100AB8EEC00ADFED300A80EE201AA4
:1076C00084ED091AE87BA97B40EA0120B082687C3E
:1076D000297C40EA012000EB80004FF6FF7101EAAF
:1076E0004000788094ED090AD4ED040AB0EE001A47
:1076F00060EE810AB4EEE00AF1EE10FA22DB94EDBE
:10770000090AD4ED080A30EE600A10EE101A084695
:10771000F8F78CFE41EC190BB0EE490AF0EE690A5D
:10772000FEF720F9B0EE408AF0EE608A9FED140B70
:1077300053EC102B51EC180BF8F7A4FE02D20520E5
:10774000E07273E794ED080ADFED0F0AB4EEE00A89
:10775000F1EE10FA01D80120207200BF66E70000A8
:1077600098000020180500209846002018470020A7
:1077700024050020D8460020E447002000007A4479
:10778000000000000000E03FCDCC4C3E00B9704747
:10779000417A094A51701146497811B90021918006
:1077A00007E005494978012903D14FF6E851024A1B
:1077B000918000BFEBE700003C77002000B97047E4
:1077C00000210C4A1278F02A01D10B4904E0094A41
:1077D00012780F2A00D10949427A00EE102AB8EE39
:1077E000400ADFED070A80EE201A81ED041A00BF7F
:1077F000E5E700009800002098460020D8460020C9
:107800000000C84200B97047002100220B4B1B78D2
:10781000F02B02D10A4A0B4905E0084B1B780F2BCD
:1078200001D1094A0949437A00EE103AB8EE400AFC
:1078300082ED040A00234B8000BFE4E7980000209B
:1078400098460020A4000020D8460020AC0000206C
:1078500010B5014601B910BD002000220F4B1B7866
:10786000F02B02D10E480F4A05E00C4B1B780F2B72
:1078700001D10D480D4A4B7A438043884FF6FF747F
:1078800004EA0323438043888C7A2343438043885C
:10789000DB4343800523D37200BFDCE79800002060
:1078A000A400002098460020AC000020D84600200C
:1078B0002DE9F84F054615B90020BDE8F88FEC68B2
:1078C000D5F808802E7C2078052801D00020F4E728
:1078D000A078617840EA012000F0FF0909F1010079
:1078E000864201DA0020E8E72079E17840EA0120C9
:1078F00000F0FF0BBBF1A10F01D00020DDE7A07964
:10790000617940EA012000F0FF0ABAF1B10F01D01D
:107910000020D2E7B01E215CF01E205C41EA00206E
:107920000090701E205C1B2801D00020C5E7E07984
:10793000F02804D0E0790F2801D00020BDE7E079DD
:1079400015490870277A394613480078FEF7BCFFBE
:10795000072F1CD2DFE807F01B04080C131B1700CD
:107960002046FFF75DFE13E02046FFF727FF0FE0FC
:107970002046FFF70BFF4046FEF716FC08E02046C6
:10798000FFF740FF04E02046FFF762FF00E000BF82
:1079900000BF012091E70000980000202DE9FE4F74
:1079A000054615B90020BDE8FE8FE81C0290EC6882
:1079B0000E300190401C009005F11A0B05F11C07D8
:1079C0003E1D05F12409217801980078814201D0FB
:1079D0000020E8E7617800980078814201D000201B
:1079E000E1E794F802A0BBF80000BAEB400F01D029
:1079F0000020D8E70AF10300C1B22046F8F742FFA1
:107A0000388094F827007978884201D00020CAE7AE
:107A100094F828003978884201D00020C3E7E07C40
:107A20000006217D40EA0140617D40EA0120A17D00
:107A300040EA010800EE108A86ED000AE07D0006AB
:107A4000217E40EA0140617E40EA0120A17E40EAB9
:107A5000010800EE108A89ED000ADFED100A9FEDA3
:107A6000100A304600F0C0FDDFED0E0A9FED0E0A51
:107A7000484600F0B9FD96ED000AF3EE080A30EE34
:107A8000C00A86ED000AF3EE070A9FED080A3046A9
:107A90000299FFF743F8012085E70000000000008D
:107AA0000000D4410000C8C20000C842CDCC4C3E0A
:107AB00010B504460CB9002010BD0948844203D11A
:107AC0002046FFF7F5FEF7E70648844202D0064855
:107AD000844203D12046FFF761FFEDE70020EBE78A
:107AE000B048002018470020E447002010B50C489B
:107AF00040880C49098888420DD002F0BDF80A4937
:107B00000968C831884206D301200849087102F08B
:107B1000B3F805490860024840880249088010BD52
:107B20003C770020C8000020C4000020B04800209E
:107B300030B500B930BDC3780479411C821C0D7882
:107B4000012D0FD1012B08D0BBEE080A80ED090AE8
:107B5000B3EE080A80ED070A16E00125057200253C
:107B60000D7011E01578012D0ED1012C08D0B3EE67
:107B7000080A80ED090ABBEE080A80ED070A03E057
:107B8000012505720025157000BFD3E72DE9F047E8
:107B90002DED048B05461DB9BDEC048BBDE8F087C7
:107BA0004FF0000900270024AE48854206D1DFF8D7
:107BB000B882DFF8B892AE4FAE4C08E0AE488542CE
:107BC00005D1DFF8B882DFF8B892AE4FAE4C20781E
:107BD000012800D1E0E7A078401CC6B2A06810B927
:107BE0004FF47A70A06095ED080AD5ED040A30EEE6
:107BF000600A10EE101A0846F8F718FC41EC190B51
:107C0000B0EE490AF0EE690AFDF7ACFEB0EE408A2C
:107C1000F0EE608A51EC180BF8F74CFCA86295ED79
:107C20000A0A10EE101A0846F8F700FC41EC190B8E
:107C3000B0EE490AF0EE690AFDF794FEB0EE408A14
:107C4000F0EE608A9FED910B53EC102B51EC180B6A
:107C5000F8F700FC7ED80020287009EB860090ED34
:107C6000000ADFED8C0A20EE200ADFED8B0A80EEA1
:107C7000201A84ED031A60780B286CD2DFE800F03C
:107C80000611285890CFCFCFCFCFBE0041F2883019
:107C9000A8F8020001F0F0FF60606078401C60709E
:107CA000BEE001F0E9FFD4E90112114488420ED38D
:107CB00042F20800A8F8020001F0DEFF711E47F84A
:107CC00021006078401C607001F0D6FF6060A7E082
:107CD00094ED030ADFED710AB4EEE00AF1EE10FA5A
:107CE00013DB701E07F1280151F8200068B901F07C
:107CF000C3FF711E07F1280242F821006078401C82
:107D0000607001F0B9FF60608AE04FF4FA71A0681A
:107D1000B0FBF1F0616800EB010A01F0ADFF8245B4
:107D200005D86078401C607001F0A6FF606077E0C5
:107D3000701E07F1280151F82000F0B1701E2831A3
:107D400051F82000C8B994ED030ADFED540AB4EEEF
:107D5000E00A01E065E062E0F1EE10FA0DD201F018
:107D60008BFF711E07F1500242F821006078401C21
:107D7000607001F081FF606052E04FF4FA71A0681A
:107D8000B0FBF1F0616800EB010A01F075FF82457C
:107D900005D86078401C607001F06EFF60603FE0C5
:107DA000701E07F1780151F82000A8B994ED030A7C
:107DB000DFED3B0AB4EEE00AF1EE10FA0CD801F068
:107DC0005BFF711E07F1780242F82100A078401C89
:107DD000A0700A20607023E04FF4FA71A068B0FB35
:107DE000F1F0616800EB010A01F046FF824504D81A
:107DF000A078401CA0700A20607011E0A0780928CB
:107E00000ADD0020A0702748007910B9012025491B
:107E100008710120207003E00020607000E000BFC6
:107E20001DE000206070A070207095ED080AD5ED6F
:107E3000040AB4EEE00AF1EE10FA01D268730AE027
:107E400095ED080AD5ED040AB4EEE00AF1EE10FA59
:107E500001DD012068730120287000F01DFC00BFC7
:107E60009AE600009846002018050020987400202B
:107E7000EC7400205C770020D84600202405002008
:107E8000C47400208C7500206C770020000000A0D6
:107E90009999C93F00007A4400007A430040CE44DB
:107EA0000000C843B04800202DE9F04F85B00446DB
:107EB00014B905B0BDE8F08F254604F1030904F1BB
:107EC0000D0804F10B0A04F1090604F10A0B701EF7
:107ED000049004F130070C300390001D0290143020
:107EE0000190002000902B48844202D12A48009043
:107EF00004E02A48844201D12948009099F8000002
:107F0000012810D10021039801600298016001202E
:107F10003070009890ED080A019880ED000A204624
:107F2000FEF7A8FE08E0307830B9012088F800009C
:107F30001C483860012028703078012828D1D4ED01
:107F4000080A94ED041A9FED180AF0EE001A11EEDB
:107F5000210AF4EEC00AF1EE10FA07D8002088F8E2
:107F60000000104838600120287011E000202870BF
:107F70003070E07A042802D101208BF80000012142
:107F80000498017001208AF8000044F620603860EF
:107F900000BF8EE79846002018470020D8460020F2
:107FA000E447002080380100CDCC4C3E70B504463B
:107FB00004B970BDE57A062D1BD2DFE805F0030792
:107FC0000B0F1216204600F0B3F813E02046FFF71F
:107FD000AFFD0FE02046FFF7D9FD0BE0FFF786FD70
:107FE00008E02046FFF760FF04E02046FFF75CFF53
:107FF00000E000BF00BF00BFDBE7000018B501468E
:108000001C4A914201D11C4808E01C4A914201D10E
:108010001B4803E01B4A914200D11B4800B918BD20
:108020000A681268C2F3401282B1027CFF2A01DBA7
:10803000002202740A685268D3B2047C621C027483
:10804000C26813556FF020020B681A600A68126844
:10805000C2F3001262B10122027000BF002200923E
:108060000A68126800920A685268009200BF00BF56
:1080700000BFD4E7A8080020E4470020EC08002057
:10808000B048002064080020184700202DE9F04186
:10809000044614B90020BDE8F081661C254604F1B1
:1080A00010072046FEF7E4F92046FFF771F80E4866
:1080B000FDF7FAFD3078012804D100203070204609
:1080C00000F044F9287801280BD12046FFF7F0FC96
:1080D0008046002028700120307000203870404613
:1080E000D9E70120D7E70000980000202DE9F047EC
:1080F00005460E460DB9BDE8F08705F12008344667
:1081000006F1040901210948F9F704FC074617B9EB
:108110000120207001E000202070207820B900208C
:10812000A9F80000C8F8000000BFE4E70010024012
:108130002DE9F04704460CB9BDE8F0872546E71C59
:1081400004F10D0804F1300604F12C094FF0000A87
:108150001248844202D1DFF848A004E0114884426A
:1081600001D1DFF844A0387801280ED144F6206010
:108170003060002028709AED080A89ED000A204638
:10818000FEF778FD0120E07206E0012088F800008B
:10819000064830600120287000BFCDE798460020D7
:1081A00018470020D8460020E4470020803801000E
:1081B00030B500B930BD0146437B00F11402141DF7
:1081C000C578012D06D1012B04D10025156025604D
:1081D0000D700CE00579012D05D123B9002515603E
:1081E00025600D7003E015680DB101250D7000BF0D
:1081F000E0E72DE9F04108B9BDE8F0810146457896
:10820000867800F11404221D00F10807C37A90ED6E
:108210000B0AB5EEC00AF1EE10FA00D1ECE7042B20
:1082200003D0052B01D0022B00D1E5E791F800C067
:10823000BCF1000F00D1DFE7D2F8008008F1010C9B
:10824000C2F800C0D4F800C0E0450DD94FF0000CD2
:1082500081F800C0C2F800C0C4F800C025B91EB93A
:108260004FF0010C87F800C000BFC5E737B586B0F6
:1082700005461446002005900490039002900121C9
:108280002846FEF751FA6423012207A92E48FAF77F
:1082900041F96423012202A92B48FAF73BF9642330
:1082A000012203A92848FAF735F96423012204A919
:1082B0002548FAF72FF96423012205A92248FAF785
:1082C00029F900212846FEF72FFA01212846FEF75A
:1082D0002BFA6423012207A91B48FAF71BF9642033
:1082E000012302AA02A900901748FAF7EAF96420CC
:1082F000012303AA03A900901348FAF7E2F96420C6
:10830000012304AA04A900900F48FAF7DAF96420BF
:10831000012305AA05A900900B48FAF7D2F99DF8A8
:10832000080000069DF80C1000EB01409DF81010AD
:1083300000EB01209DF8141008442060002128461D
:10834000FEF7F2F909B030BD9C0500202DE9F05F81
:1083500005460DB9BDE8F09FA86800B9FAE71D48C9
:10836000854200D1F6E705F12809AC6805F1110A4C
:1083700005F1120B05F1180705F11A083E1D9AF8D0
:10838000000004F8010B9BF8000004F8010B78785A
:1083900004F8010B387804F8010B98F8010004F890
:1083A000010B98F8000004F8010B0621A868F8F703
:1083B00069FA3080707804F8010B307804F8010B0A
:1083C0004FF6FF7308224846A968FBF7A0FE00BFDE
:1083D000C0E70000B048002010B50446204600F079
:1083E0003DF8204600F004F8204600F095F810BD56
:1083F00070B5054605B970BD05F10C04661C3078F2
:1084000088B92078F02805D1012211031148F9F725
:1084100093FA1DE020780F281AD1012208210E4876
:10842000F9F78AFA14E03078012811D12078F02881
:1084300006D100224FF480510648F9F77DFA07E093
:1084400020780F2804D1002208210348F9F774FA94
:1084500000BFD0E7000C0240001802402DE9F041B7
:1084600004460CB9BDE8F08104F10C05264604F180
:1084700034073078012828D100202449096848624F
:108480002248FAF725FB2878F0280DD100224FF476
:1084900000511F48F9F750FA1C4938680968C86349
:1084A00008211A48FBF7EEF928780F282BD1002273
:1084B00004211848F9F740FA144938680968086433
:1084C0000C211248FBF7DEF91DE03078D8B9287886
:1084D000F02809D108210D48FBF7D8FA01225103F1
:1084E0000B48F9F729FA0BE028780F2808D10C215E
:1084F0000648FBF7CBFA012204210648F9F71CFADB
:108500000248FAF739FB00BFACE70000440700203F
:10851000000C0240001802402DE9F05F04460CB93F
:10852000BDE8F09F254604F10C06D4F83090D4F84D
:1085300034A01648B0FBF9F0471E0AFB07F064218F
:10854000B0FBF1F804F1380B2C46287800B9E7E7C6
:1085500030785A467521FFF789FE00BF0C48006845
:10856000C7620B48C76000BF3078F02804D10848C4
:108570000068C0F83C8006E030780F2803D104483A
:108580000068C0F8408000BFCAE7000040420F000A
:108590004407002070B5044604B970BD04F10C0511
:1085A0002E1D95ED000AF1EE040AB4EEE00AF1EE9C
:1085B00010FA11DB95ED000AF2EE040AB4EEE00ABF
:1085C000F1EE10FA08D8308806490968486300219E
:1085D0000448FBF7D1F803E000210248FBF702FA58
:1085E00000BFDAE71C08002090ED001AB4EEC01AB4
:1085F000F1EE10FA02DD80ED000A08E090ED001ABD
:10860000B4EEE01AF1EE10FA01D2C0ED000A7047A4
:1086100037B584B005461446E0B20390C4F3072092
:108620000290C4F307400190200E009001212846DB
:10863000FEF77AF80A2000F09FFE9DF8140040F043
:10864000800005906423012205A91248F9F762FF12
:108650006423012269460F48F9F75CFF6423012275
:1086600001A90C48F9F756FF6423012202A9094821
:10867000F9F750FF6423012203A90648F9F74AFFDE
:1086800000212846FEF750F80A2000F075FE07B0DA
:1086900030BD00009C05002010B5002016E0002130
:1086A00010E0002200EB80030A4C04EBC30343F804
:1086B000212000EB8003084C04EBC30343F8212086
:1086C0004A1CD1B20A29ECDB411CC8B20428E6DB03
:1086D00010BD0000EC7400208C75002070B50546BC
:1086E00005B970BD05F12004206818B12068401E4E
:1086F000206003E024212846F7F70EFE00BFF0E7D4
:10870000F9F732F9FCF7F4FBFBF7BCFFFBF70EFFC0
:10871000FCF7CEFAFCF7E8FAFCF702FBFBF764FD86
:10872000FBF758FEFBF7DCFEFBF710FEFCF7CCF97D
:10873000FCF708FAFCF73AF9FCF742FAFCF712F9F1
:10874000FCF756F9FCF788F9FCF784FAFBF73AFFD7
:1087500000F015F800BFFEE701460020842901D093
:10876000CA1C1044704770B5044625460DB1294611
:1087700000E00121084600F0FFFD002070BD10B5AB
:1087800000F056FE002010BD10B50446606820B110
:108790000120616800F0B7FF10BD012000F0A2FFCA
:1087A000FAE7F8B504460D46606860B1012D08D1BE
:1087B00003200090002211460120636800F0E5FFCD
:1087C000F8BD0020FCE7012D0ED10322002101207D
:1087D00000F0AEFF06462EB100231A461946304679
:1087E00001F090F83046EBE70020E9E77FB504465A
:1087F0000D46606998B1A06988B1B4F90800FFF727
:10880000ABFF0646D4E90510CDE9006102902B4686
:108810002269D4E9001001F0C1F9039013E0B4F922
:108820000800FFF799FF064603A8CDE90060238AF8
:108830009AB22B46D4E9001001F07EF9012802D04B
:10884000002004B070BD0398FBE700002DE9F04163
:1088500005460E461C4807681C480068001D00F0CD
:1088600087FC50B91948006890F82C100120884006
:1088700017490968814316480160681C38B936B148
:1088800012480168091D134800F0BCFC1AE07C196D
:108890000E4800684460BC4207D20C480168091DBC
:1088A0000D48006800F094FC0CE008480168091DC0
:1088B0000A48006800F08CFC09480068844201D234
:1088C00007480460BDE8F08144000020300000202B
:1088D00048000020540A0020380000203400002006
:1088E0006000002010B5044600F098FC23480068A2
:1088F000401C224908602248006840B920480460B2
:108900000846006801280DD100F0A0F90AE01D48D2
:10891000006838B91A480068C06AE16A884201D81C
:108920001748046018480068401C1749086094F80C
:108930002C10012088401549096808431349086034
:10894000E16A01EB8101124A02EB8100211D00F076
:1089500059FC00F08DFC0B48006868B108480068BD
:10896000C06AE16A884207D24FF080500949086026
:10897000BFF34F8FBFF36F8F10BD0000400000208A
:10898000300000204C0000205C0000204800002047
:108990007809002004ED00E010B516E000F03EFC80
:1089A0000C48C068C468201D00F0E2FB0A4800685B
:1089B000401E0949086009480068401E07490860D0
:1089C00000F056FC204600F04AF8044800680028F1
:1089D000E4D110BD400A0020400000203C000020EF
:1089E0002DE9F04104460F4615464FF00008A66BEE
:1089F000206C48B9206800282CD1A06801F0E6F965
:108A000080460020A06025E07DB93946226C606870
:108A1000F7F769FC216C606808446060D4E90101E3
:108A2000884217D32068606014E03946226CE06801
:108A3000F7F759FC216CE068411AE1602168E068B1
:108A4000884203D2216CA068411AE160022D01D155
:108A500006B1761E701CA0634046BDE8F08110B5DB
:108A6000044694F8510030B9206B00F01FFC2046FA
:108A700000F01CFC1AE094F85100012803D12046B4
:108A800000F014FC12E094F85100022801D10120FA
:108A900000E0002050B900BF502080F31188BFF3E0
:108AA0004F8FBFF36F8F00BF00BFFEE710BD000008
:108AB00030B54FF47053174800F007042CB1C01DB7
:108AC00020F00700134C041B1B1B0246124C2260B3
:108AD0000024114D6C60D018083820F007000F4CAE
:108AE000206000240D4D2D686C600C4D2D682C60AD
:108AF0001146441A4C60094C24680C60084D4C68BF
:108B00002C60084D4C682C604FF00044064D2C60E2
:108B100030BD0000680A00206C00002074000020B6
:108B20007C000020780000208800002000BFFFF7B4
:108B300033FF064800680128F9D94FF080500449F6
:108B40000860BFF34F8FBFF36F8FF0E77809002005
:108B500004ED00E010B5044654B10020A060206090
:108B60000021E16000231A461946204600F0CAFEA3
:108B700010BD2DE9F04106460D4617469846069C65
:108B80000DB9246000E02760E663256401212046DA
:108B900000F06CFEBDE8F0812DE9FF5F81460E46D6
:108BA0009246DDE90E7B109CAAF10100216B01EBDE
:108BB000800828F0070808F0070008B9012000E045
:108BC000002050B900BF502080F31188BFF34F8FB1
:108BD000BFF36F8F00BF00BFFEE786B1002507E03F
:108BE000715D04F134004155705D00B902E06D1C07
:108BF000102DF5D300BF00214320015502E00020D5
:108C000084F83400072F00D30627E762676400204A
:108C1000A064201D00F0D9FA04F1180000F0D5FA84
:108C20002461C7F10700A06164620020E06484F859
:108C3000500049464046039A00F0A0F92060BBF17D
:108C4000000F01D0CBF80040BDE8FF9F10B5002415
:108C500007E004EB84010F4A02EB810000F0A8FA60
:108C6000641C072CF5D30C4800F0A2FA0B4800F066
:108C70009FFA0B4800F09CFA0A4800F099FA0A485B
:108C800000F096FA04480949086004480849086059
:108C900010BD000078090020040A0020180A0020F6
:108CA0002C0A0020400A0020540A00203400002032
:108CB0003800002010B50146164800E0006803683F
:108CC0008B42FBD30246436813448B4204D1436872
:108CD0004C682344436001460A464B6813440468C9
:108CE000A34211D10C4C03682468A34208D04B68FE
:108CF0000468646823444B6003681B680B6005E0EC
:108D0000054B1B680B6001E003680B60884200D0D4
:108D1000016010BD6C0000207400002070B5054695
:108D200000F07CFAA86BE96B884201D1012400E0D5
:108D3000002400F09DFA204670BD00000A49096831
:108D4000096809B9012100E0002121B14FF0FF318C
:108D5000064A116006E004490968C968C868034A00
:108D6000416811607047000034000020600000205E
:108D70000E480068401C08B9012000E0002050B9EE
:108D800000BF502080F31188BFF34F8FBFF36F8F68
:108D900000BF00BFFEE700BF502080F31188BFF383
:108DA0004F8FBFF36F8F00BF00BFFEE78C00002026
:108DB00070B5044600F032FA94F9455010E0606A4C
:108DC00008B9012000E0002038B904F1240001F0C6
:108DD00061F818B100F00AFB00E003E0681E45B23C
:108DE000002DECDC00BFFF2084F8450000F040FAC5
:108DF00000F014FA94F9445010E0206908B90120F9
:108E000000E0002048B904F1100001F043F808B177
:108E100000F0ECFA681E45B200E001E0002DECDC49
:108E200000BFFF2084F8440000F022FA70BD00006B
:108E30002DE9F04104464FF0000800F051FB49488D
:108E4000006808B9FFF734FE474800682040002852
:108E500070D1D4B1083404F00700B0B104F00700B9
:108E6000C0F10800044404F0070008B9012000E044
:108E7000002050B900BF502080F31188BFF34F8FFE
:108E8000BFF36F8F00BF00BFFEE7002C52D0374802
:108E9000006884424ED8364E3046056801E02E46C2
:108EA0002D686868A04202D228680028F7D12D48B2
:108EB000006885423ED0306800F1080828683060BC
:108EC0006868001B102819D92F1907F0070008B986
:108ED000012000E0002050B900BF502080F311882D
:108EE000BFF34F8FBFF36F8F00BF00BFFEE768680F
:108EF000001B78606C603846FFF7DCFE1B49686831
:108F00000968081A1949086008460068194909687B
:108F1000884203D2154800681649086012496868FB
:108F20000968084368600020286013480068401CF6
:108F30001149086000F0FAFF08F0070008B90120A5
:108F400000E0002050B900BF502080F31188BFF32B
:108F50004F8FBFF36F8F00BF00BFFEE74046BDE8F5
:108F6000F0810000740000208800002078000020BC
:108F70006C0000207C00002080000020001F4FF0CB
:108F800080730360001F21F001030360001F054B85
:108F9000036014380260001F6FF002030360203882
:108FA00070470000718D00080F48FEF723FA0F4844
:108FB000FEF720FA0E48FEF71DFA00BF0D480078B4
:108FC000F02803D10848FFF761F806E00948007867
:108FD0000F2802D10548FFF759F80548FFF756F862
:108FE0000120FFF7C0FBE9E718470020E447002015
:108FF000B0480020980000202A48FEF7BBF92A4814
:10900000FEF7B8F929492A48FEF794F929492A4870
:10901000FEF790F9012251032848F8F78DFC012250
:1090200004212748F8F788FC012251022348F8F769
:1090300083FC2448FEF7CAFA0A2000F09DF9224872
:10904000FEF7C4FA00BF21480078F0280DD10020B7
:109050001D4908700846FFF7BFF916491648FDF785
:1090600073FC1848FDF7D8FA10E0184800780F286C
:109070000CD10020134908700846FFF7ADF90B49E1
:109080000B48FDF761FC1048FDF7C6FA1048FDF7E4
:10909000A5FA4FF4FA70FDF775FA0A20FFF763FBA3
:1090A000D1E70000F47600201877002080460020E9
:1090B000B406002068460020FC060020000C024098
:1090C0000018024098460020D84600209800002052
:1090D0003C7700201248FEF7D1F81248FEF7CEF890
:1090E0001148FEF701F91148FEF7FEF81048FEF7A7
:1090F0008DF81048FEF78AF800BF0B490848FCF7C6
:10910000F3FC0A490748FCF7EFFC0948FDF7D8F9DA
:109110000848FDF7D5F94FF47A70FFF724FBECE728
:10912000CC4F0020E44F0020FC4F002028500020AE
:10913000A4000020AC000020FEF780F80A48FEF7EB
:109140003DFA0A48FEF73AFA00BFFDF7ADFEFDF71B
:1091500095FE0548FDF776FA0448FDF773FA0120FD
:10916000FFF701FBF1E700001805002024050020AF
:1091700001460A69D1E901309860D1E901035860DC
:109180005068884201D188685060002008611068EA
:10919000401E106010687047034B0360034B0B6068
:1091A0008023136070470000CC00002020010020C5
:1091B00000F1080141604FF0FF31816000F10801CA
:1091C000C1600161002101607047002101617047A9
:1091D00010B502460B685C1C0CB9106907E002F17F
:1091E000080000E04068446824689C42FAD944685A
:1091F0004C604C68A160886041600A611468641C1E
:10920000146010BD42684A6093688B60936859602F
:109210009160086103685B1C0360704700BF5020C9
:1092200080F31188BFF34F8FBFF36F8F00BF0E48DD
:109230000068401C0C49086008460068012812D1EB
:109240000A480068C0B208B9012000E0002050B907
:1092500000BF502080F31188BFF34F8FBFF36F8F93
:1092600000BF00BFFEE770478C00002004ED00E067
:109270000D48006850B900BF502080F31188BFF33B
:109280004F8FBFF36F8F00BF00BFFEE70648006837
:10929000401E054908600846006820B9002080F398
:1092A000118800BF00BF70478C00002070B50646D3
:1092B0003546002E44D0083D2C4622496068096896
:1092C000084008B1012000E0002050B900BF502044
:1092D00080F31188BFF34F8FBFF36F8F00BF00BFC4
:1092E000FEE7206808B9012000E0002050B900BF67
:1092F000502080F31188BFF34F8FBFF36F8F00BFF3
:1093000000BFFEE70F49606809680840C0B12068E7
:10931000B0B90C49606809688843606000F0E0F803
:109320000949606809680844074908602046FFF752
:10933000C1FC06480068401C0449086000F0F6FDC6
:1093400070BD00008800002078000020840000200C
:1093500000204FF0E02108618861064800684FF462
:109360007A71B0FBF1F0401E4FF0E0214861072018
:10937000086170472C00002070B504460025D4B168
:109380001248006808B9012000E0002050B900BF71
:10939000502080F31188BFF34F8FBFF36F8F00BF52
:1093A00000BFFEE700F09CF800212046FFF74EFAD0
:1093B00000F0BCFD05463DB94FF0805004490860FF
:1093C000BFF34F8FBFF36F8F70BD000068000020A8
:1093D00004ED00E003490968016003490968416040
:1093E000704700005800002044000020012001497F
:1093F000086070475400002070B504460D4654B90B
:1094000000BF502080F31188BFF34F8FBFF36F8FE1
:1094100000BF00BFFEE70548016818312046FFF78E
:10942000D7FE01212846FFF711FA70BD3000002059
:1094300010B586B000200590049003AA04A905A8E1
:10944000FFF7AAFE0022DDE904101346CDE9002152
:1094500002901CA11D48039A00F0A0FB1C49086063
:109460000846006808B1012400E00024012C15D151
:1094700000BF502080F31188BFF34F8FBFF36F8F71
:1094800000BF4FF0FF301349086001201249086007
:1094900000201249086000F071F810E0601C08B16B
:1094A000012000E0002050B900BF502080F3118857
:1094B000BFF34F8FBFF36F8F00BF00BFFEE706B053
:1094C00010BD000049444C45000000002D8B0008F1
:1094D00064000020600000204C00002044000020B8
:1094E00002480068401C014908607047680000207D
:1094F0001D48006818B101201C49086032E00020B6
:109500001A4908601A480068B0FA80F0C0F11F01DB
:1095100001EB8100174A52F8200008B1012000E059
:10952000002050B900BF502080F31188BFF34F8F47
:10953000BFF36F8F00BF00BFFEE701EB81020D4B51
:1095400003EB820042685268426000F108024368FF
:10955000934202D14268526842604268D268064B28
:109560001A6000BF7047000068000020540000200F
:109570004800002078090020300000201CB5524827
:1095800000685249884201D0012000E0002050B913
:1095900000BF502080F31188BFF34F8FBFF36F8F50
:1095A00000BF00BFFEE7484800684849491E88429E
:1095B00001D0012000E0002050B900BF502080F30E
:1095C0001188BFF34F8FBFF36F8F00BF00BFFEE75F
:1095D0003F49084600780190FF200A46107008466F
:1095E000007800909DF8000000F0F0009DF8002049
:1095F000904201D1012000E0002050B900BF50206E
:1096000080F31188BFF34F8FBFF36F8F00BF00BF90
:10961000FEE79DF8000000F050002E4A1070072071
:109620002D4A106009E02C480068401E2A4A10604C
:109630009DF800004006000E00909DF8000000F02C
:1096400080008028EFD024480068C0F1070004287B
:1096500001D1012000E0002050B900BF502080F36C
:109660001188BFF34F8FBFF36F8F00BF00BFFEE7BE
:10967000194800680002184A10601046008800F47B
:10968000E0601060124A019810700F4820300068A6
:1096900040F470000C49203108600846006840F032
:1096A00070400860FFF754FE00200C490860F6F790
:1096B0009BFD0B48006840F0404009490860F6F700
:1096C0007FFD00201CBD000000ED00E071C20F41D5
:1096D00000E400E090000020940000208C000020B6
:1096E00034EF00E02DE9F041044601260027224630
:1096F0000021012000F01CF805462846FFF72AFA51
:109700002846BDE8F0812DE9F84304460D460127BF
:109710004FF000082B46002211460120009400F073
:1097200034F806463046FFF715FA3046BDE8F883B0
:109730002DE9F84305460E4617460DB1012000E01D
:10974000002050B900BF502080F31188BFF34F8F25
:10975000BFF36F8F00BF00BFFEE705FB06F808F1FF
:109760004800FFF765FB044664B1A14609F14809CA
:10977000002084F846003B464A463146284600947D
:10978000FFF7F7F92046BDE8F8832DE9F843804656
:109790000E4617461D46DDF82090B8F1000F01D0A7
:1097A000012000E0002050B900BF502080F3118854
:1097B000BFF34F8FBFF36F8F00BF00BFFEE70DB148
:1097C000012000E0002050B900BF502080F3118834
:1097D000BFF34F8FBFF36F8F00BF00BFFEE707B12E
:1097E0000EB1012000E0002050B900BF502080F3EE
:1097F0001188BFF34F8FBFF36F8F00BF00BFFEE72D
:1098000007B90EB9012000E0002050B900BF502078
:1098100080F31188BFF34F8FBFF36F8F00BF00BF7E
:10982000FEE7482000900098482801D1012000E080
:10983000002050B900BF502080F31188BFF34F8F34
:10984000BFF36F8F00BF00BFFEE700BF2C464CB1D7
:10985000012084F846004B463A4631464046009483
:10986000FFF787F92046BDE8F883000070B505468C
:109870000E462C4654B900BF502080F31188BFF328
:109880004F8FBFF36F8F00BF00BFFEE7FFF7C6FC2F
:10989000D4E90F12206801FB0200A0600020A06341
:1098A00020686060E06B401E226C216800FB0211A2
:1098B000E160FF2084F8440084F845009EB92069E7
:1098C00008B9012000E00020A8B904F1100000F060
:1098D000E1FA80B14FF0805009490860BFF34F8F23
:1098E000BFF36F8F07E004F11000FFF761FC04F194
:1098F0002400FFF75DFCFFF7BBFC012070BD0000FA
:1099000004ED00E02DE9FF4383B0064688461D467E
:109910004FF00009344654B900BF502080F311883D
:10992000BFF34F8FBFF36F8F00BF00BFFEE7B8F1EB
:10993000000F01D1206C08B9012000E0002050B9CF
:1099400000BF502080F31188BFF34F8FBFF36F8F9C
:1099500000BF00BFFEE7022D02D1E06B012801D15C
:10996000012000E0002050B900BF502080F3118892
:10997000BFF34F8FBFF36F8F00BF00BFFEE700F054
:109980006BF908B9059808B9012000E0002050B92A
:1099900000BF502080F31188BFF34F8FBFF36F8F4C
:1099A00000BF00BFFEE700BFFFF738FCA06BE16B14
:1099B000884201D3022D28D12A4641462046FFF78E
:1099C0000FF80746606A08B9012000E0002068B976
:1099D00004F1240000F05EFA88B14FF08050324963
:1099E0000860BFF34F8FBFF36F8F08E03FB14FF0B8
:1099F00080502D490860BFF34F8FBFF36F8FFFF783
:109A000037FC012007B0BDE8F083059818B9FFF7CF
:109A10002FFC0020F6E7B9F1000F04D101A8FFF7F1
:109A2000D9FC4FF00109FFF723FCFFF759FDFFF7C1
:109A3000F5FB94F94400401C10B9002084F8440060
:109A400094F94500401C10B9002084F84500FFF748
:109A50000FFC05A901A800F029F8F0B92046FFF78E
:109A60005DF9A0B104F110000599FFF7C5FC20468F
:109A7000FFF79EF900F05AFA002895D14FF0805078
:109A800009490860BFF34F8FBFF36F8F8CE7204603
:109A9000FFF78EF900F04AFA86E72046FFF788F9CB
:109AA00000F044FA0020ADE704ED00E070B5054693
:109AB0000C4655B900BF502080F31188BFF34F8F7B
:109AC000BFF36F8F00BF00BFFEE754B900BF502047
:109AD00080F31188BFF34F8FBFF36F8F00BF00BFBC
:109AE000FEE7FFF79BFB124802686868131A2068BC
:109AF000401C08B9002617E00E492868096888420A
:109B000004D06868904201D801260DE02068984290
:109B100007D92068C01A20602846FFF75BFC0026A2
:109B200002E0002020600126FFF7A2FB304670BD56
:109B300044000020580000202DE9FF4F85B08046EA
:109B400089461746DDE912ABB800FFF771F9064602
:109B500056B15420FFF76CF904460CB1266304E0BB
:109B60003046FFF7A3FB00E000248CB1002084F80E
:109B70005100CDE900ABCDE902403A4649464046A6
:109B8000089BFFF709F82046FEF7ACFE012501E02F
:109B90004FF0FF35284609B0BDE8F08F2DE9F04FB2
:109BA00085B00746884691469A46DDE90EB6109C78
:109BB0000EB1012000E0002050B900BF502080F31A
:109BC0001188BFF34F8FBFF36F8F00BF00BFFEE759
:109BD0000CB1012000E0002050B900BF502080F3FC
:109BE0001188BFF34F8FBFF36F8F00BF00BFFEE739
:109BF000542003900398542801D1012000E0002054
:109C000050B900BF502080F31188BFF34F8FBFF3CE
:109C10006F8F00BF00BFFEE700BFB4B1AEB12546F5
:109C20002C462E63022085F85100002004A95346DB
:109C30004A46CDE900B1CDE9025041463846FEF72B
:109C4000ABFF2846FEF74EFE01E00020049004988A
:109C500005B0BDE8F08F00000549096809B9012089
:109C600005E00449096809B9022000E000207047B6
:109C70004C0000206800002001490868704700007F
:109C8000440000202DE9F0414FF0000844480068EE
:109C900000287CD143480068451C4248056015BB3C
:109CA00041480068006808B9012000E0002050B970
:109CB00000BF502080F31188BFF34F8FBFF36F8F29
:109CC00000BF00BFFEE738480768384800683649DB
:109CD00008603648076036480068401C3449086010
:109CE000FFF72CF800BF3348006885423CD300BF23
:109CF0002D480068006808B9012000E0002020B16C
:109D00004FF0FF302B4908602DE027480068C068FD
:109D1000C4686668B54202D22648066023E0201D6A
:109D2000FFF726FAA06A18B104F11800FFF720FA2D
:109D300094F82C10012088401F49096808431E49E7
:109D40000860E16A01EB81011C4A02EB8100211DE0
:109D5000FFF758FA1A49E06A0968C96A8842C7D306
:109D60004FF00108C4E700BF15480068C06A00EB67
:109D70008000124951F82000012801D94FF0010854
:109D80001048006808B14FF0010805E0FFE70E48F1
:109D90000068401C0C4908604046BDE8F0810000A6
:109DA000680000204400002034000020380000201B
:109DB00058000020600000204800002078090020A2
:109DC00030000020540000205000002070B50546EF
:109DD0002C460026002D55D02B480068844201D126
:109DE000012000E0002050B900BF502080F311880E
:109DF000BFF34F8FBFF36F8F00BF00BFFEE7A06CB4
:109E000050B900BF502080F31188BFF34F8FBFF3CC
:109E10006F8F00BF00BFFEE7A06C401EA064616CA6
:109E2000E06A88422ED0A06C60BB201DFFF7A0F92D
:109E300078B9E06A00EB8000144951F8200040B97D
:109E400094F82C100120884011490968814310487A
:109E50000160606CE062E06AC0F10700A06194F804
:109E60002C10012088400A49096808430849086005
:109E7000E16A01EB8101054A02EB8100211DFFF738
:109E8000C1F90126304670BD30000020780900205D
:109E90004800002070B50646F068C46854B900BF99
:109EA000502080F31188BFF34F8FBFF36F8F00BF37
:109EB00000BFFEE704F11800FFF75AF915480068E3
:109EC000A8B9201DFFF754F994F82C100120884000
:109ED00011490968084310490860E16A01EB8101F2
:109EE0000E4A02EB8100211DFFF78CF904E004F11A
:109EF00018010B48FFF786F90A49E06A0968C96A40
:109F0000884204D9012501200749086000E00025A6
:109F1000284670BD68000020480000207809002015
:109F20002C0A0020300000205400002070B50024CE
:109F300000263648006850B900BF502080F31188D1
:109F4000BFF34F8FBFF36F8F00BF00BFFEE7FFF778
:109F500065F92E480068401E2C49086008460068D4
:109F600000284FD12A48006800284BD024E0294817
:109F7000C068C46804F11800FFF7FAF8201DFFF765
:109F8000F7F894F82C100120884023490968084309
:109F900021490860E16A01EB8101204A02EB81005E
:109FA000211DFFF72FF91E49E06A0968C96A884236
:109FB00002D301201B4908601648006808B9012037
:109FC00000E000200028D2D00CB1FEF7B7FE164802
:109FD000056865B100BFFFF755FE10B101201149BA
:109FE00008606D1E002DF6D100200F4908600D4855
:109FF000006838B1012630070C490860BFF34F8F65
:10A00000BFF36F8FFFF734F9304670BD6800002052
:10A01000400000202C0A0020480000207809002081
:10A0200030000020540000205000002004ED00E02B
:10A0300008A10008A54E0008000000000000000074
:10A0400080000000000000000000000014A10008D3
:10A05000A98F0008FDFF00000000000000080000BC
:10A060000000000000000000F8A00008399100087E
:10A07000FDFF000000000000800000000000000064
:10A080000000000020A10008F98F0008FDFF00007B
:10A0900000000000000200000000000000000000BE
:10A0A000E8A00008D5900008FDFF000000000000B7
:10A0B00080000000000000000000000000061016F4
:10A0C000000610160000000000000000010203045A
:10A0D000060708090000000001020304E784D3D644
:10A0E000B47677C4F7F600007461736B5F646973CC
:10A0F000706C61795F7265007461736B5F67657422
:10A100005F7377697463680064656661756C745425
:10A1100061736B007461736B5F636F6D00000000AF
:10A120007461736B5F6374725F6D6F746F72000044
:10A1300050A1000800000020CC0000007859000861
:10A140001CA20008CC000020B47A00008859000846
:10A1500000000000000000000000000000000000FF
:10A160000000000000000000000000005800000097
:10A170000000000010000000010000000024F400B6
:10A1800000000000000000000000000000000000CF
:10A1900000000000000000000000000000000000BF
:10A1A00000000000000000000000000000000000AF
:10A1B000000000000000000000000000000000009F
:10A1C000000000000000000000000000000000008F
:10A1D000000000000000000000000000AAAAAAAAD7
:10A1E0000000000000000000F0000000000000007F
:10A1F000000000000000000000000000000000005F
:10A20000000000000000000000000000000000004E
:0CA2100000000000000000000000000042
:040000050800018965
:00000001FF
